:0200000480007A
:100000007310403073104034F32740F181CB73F00C
:1000100007307310403073005010F5BFB711004027
:1000200093810180B7070440938707003E810A82CD
:1000300073100134A52200000841B7170080938790
:1000400007001D8D828037070080AA951307073DA2
:100050006315B5001345F6FF82808347050093566C
:1000600086000505B18F93F7F70FB3C7E7209043DC
:10007000358EF9BFB706DEC0814737D7003091060D
:100080000568B70502003E9508C374C3010001006E
:100090000100010001003047058A75FEC297E39414
:1000A000B7FE82803715028013050500E1B73708D7
:1000B000DEC02E87AA86330EC5003D43B7D7003079
:1000C0000908B308DE406369130793574600415798
:1000D000B387E7023E9655C21D8D9D8D1C4141118F
:1000E0003EC05C413EC21C453EC45C453EC68147A5
:1000F000B386F50083C606003307F10085072300A9
:10010000D700E317F6FEB7D7003088C30247D8C33D
:10011000124798C72247D8C7324798CB3707DEC067
:100120000907F8C301000100010001000100B84700
:10013000058B75FF4101828094C38328070023A2A9
:1001400017018328470023A417018328870023A6CB
:1001500017018328C70023A8170123A20705010060
:10016000010001000100010083A8870493F8180032
:10017000E39C08FEC1064107A9B78280B717028039
:100180009387070033C5A7201DB79041371700801C
:10019000914713070700998F3E9611BF397106DE0C
:1001A00022DC26DA4AD84ED652D456D25AD05ECE67
:1001B00062CCB7E7003003D707000146136707405A
:1001C0002390E70003D70701136707402398E70050
:1001D00037270028545F9396E6289396F62854DF35
:1001E0008356470393E60608231AD7024567130789
:1001F000171223AEE70A054798DBD85F945B930597
:10020000C6F90D8B8D8A99C16398E6143767C10FC3
:10021000B7E7003013077710B8CB23AA07041307FA
:100220002003B8CFB84B1377F7F913670702B8CBA1
:10023000B853058B75DFB84BB7D600303706F1FFE2
:10024000659B13674700B8CBF8467D16718F13176F
:10025000072913171729F8C6F84637E60030136741
:100260002700F8C6094798DB8146585E1C5A9385DB
:10027000C6F90D8B8D8B99C16312F70EB70B0080F9
:1002800083A90B7D371A008013040A00B704060007
:1002900037190480FD57A294B71A0080130909008A
:1002A0006390F90C03AB0A00B3058B403387F5006C
:1002B000B7070200A91763E5E70A4E862285613376
:1002C0002AC02A8C41468A855A854EC24EC44EC6E3
:1002D000F93B83270B00639587092685613BA2853F
:1002E00026856535B7B71234938757A541468A8569
:1002F00013850B7D3EC0653BB7090200A919130C9D
:100300000A00370B0400B70B060003AA0A00B30566
:100310008A409387F5FF63EBF9007D5662852533AC
:1003200083270A006394A700EF00D04D032A090039
:10033000B3058A409387F5FF63E7F9067D564A8542
:100340001933B3074B019C43639FA70422851D33D8
:10035000CA8522851D3D55BF050645B5850631B7C1
:10036000370B0200B309640183AB09009307ABFEAE
:10037000B3858B401387F5FFE3E0E7F87D564E85A4
:10038000D9315E9B83270B00E398A7F64A85DD31C0
:10039000A2854A85DD3B2285F1392285CE85F5335C
:1003A0004E85C93991BF03AA0400B3058A409387DB
:1003B000F5FF63EEF9007D5626857131B3874B0159
:1003C0009C436396A70022857531A68559B701A085
:1003D00000000000963007772C610EEEBA510999A3
:1003E00019C46D078FF46A7035A563E9A395649EFF
:1003F0003288DB0EA4B8DC791EE9D5E088D9D29723
:100400002B4CB609BD7CB17E072DB8E7911DBF907E
:100410006410B71DF220B06A4871B9F3DE41BE84A2
:100420007DD4DA1AEBE4DD6D51B5D4F4C785D383FE
:1004300056986C13C0A86B647AF962FDECC9658AA2
:100440004F5C0114D96C0663633D0FFAF50D088DFE
:10045000C8206E3B5E10694CE44160D5727167A2A2
:10046000D1E4033C47D4044BFD850DD26BB50AA5FE
:10047000FAA8B5356C98B242D6C9BBDB40F9BCAC22
:10048000E36CD832755CDF45CF0DD6DC593DD1AB7E
:10049000AC30D9263A00DE518051D7C81661D0BFA2
:1004A000B5F4B42123C4B3569995BACF0FA5BDB8FE
:1004B0009EB802280888055FB2D90CC624E90BB1A2
:1004C000877C6F2F114C6858AB1D61C13D2D66B6FE
:1004D0009041DC760671DB01BC20D2982A10D5EF62
:1004E0008985B1711FB5B606A5E4BF9F33D4B8E8BE
:1004F000A2C9077834F9000F8EA8099618980EE162
:10050000BB0D6A7F2D3D6D08976C6491015C63E6BD
:10051000F4516B6B62616C1CD83065854E0062F2E1
:10052000ED95066C7BA5011BC1F4088257C40FF53D
:10053000C6D9B06550E9B712EAB8BE8B7C88B9FC61
:10054000DF1DDD62492DDA15F37CD38C654CD4FBBD
:100550005861B24DCE51B53A7400BCA3E230BBD461
:1005600041A5DF4AD795D83D6DC4D1A4FBF4D6D3BD
:100570006AE96943FCD96E34468867ADD0B860DA61
:10058000732D0444E51D03335F4C0AAAC97C0DDDBD
:100590003C710550AA41022710100BBE86200CC9E1
:1005A00025B56857B3856F2009D466B99FE461CE3D
:1005B0000EF9DE5E98C9D9292298D0B0B4A8D7C761
:1005C000173DB359810DB42E3B5CBDB7AD6CBAC0BD
:1005D0002083B8EDB6B3BF9A0CE2B6039AD2B174D9
:1005E0003947D5EAAF77D29D1526DB048316DC7335
:1005F000120B63E3843B64943E6A6D0DA85A6A7AD9
:100600000BCF0EE49DFF099327AE000AB19E077D34
:1006100044930FF0D2A3088768F2011EFEC2066958
:100620005D5762F7CB67658071366C19E7066B6EB4
:10063000761BD4FEE02BD3895A7ADA10CC4ADD67D8
:100640006FDFB9F9F9EFBE8E43BEB717D58EB06034
:10065000E8A3D6D67E93D1A1C4C2D83852F2DF4FD8
:10066000F167BBD16757BCA6DD06B53F4B36B24834
:10067000DA2B0DD84C1B0AAFF64A0336607A0441D8
:10068000C3EF60DF55DF67A8EF8E6E3179BE694634
:100690008CB361CB1A8366BCA0D26F2536E2685258
:1006A00095770CCC03470BBBB91602222F260555B4
:1006B000BE3BBAC5280BBDB2925AB42B046AB35CD8
:1006C000A7FFD7C231CFD0B58B9ED92C1DAEDE5B34
:1006D000B0C2649B26F263EC9CA36A750A936D0218
:1006E000A906099C3F360EEB856707721357000574
:1006F000824ABF95147AB8E2AE2BB17B381BB60C98
:100700009B8ED2920DBED5E5B7EFDC7C21DFDB0BF3
:10071000D4D2D38642E2D4F1F8B3DD686E83DA1F17
:10072000CD16BE815B26B9F6E177B06F7747B71873
:10073000E65A0888706A0FFFCA3B06665C0B011117
:10074000FF9E658F69AE62F8D3FF6B6145CF6C1673
:1007500078E20AA0EED20DD75483044EC2B3033917
:10076000612667A7F71660D04D476949DB776E3E73
:100770004A6AD1AEDC5AD6D9660BDF40F03BD83797
:1007800053AEBCA9C59EBBDE7FCFB247E9FFB530F3
:100790001CF2BDBD8AC2BACA3093B353A6A3B42417
:1007A0000536D0BA9306D7CD2957DE54BF67D92373
:1007B0002E7A66B3B84A61C4021B685D942B6F2A17
:1007C00037BE0BB4A18E0CC31BDF055A8DEF022D73
:1007D000FFFFFFFFFFFFFFFFFFFFFFFFFFFFFFFF29
:1010000030A80080B711004093810180B7170138E4
:1010100023A40700B71700809387073273905730D7
:10102000F327103093F7870291C7896773A00730C1
:1010300073103000B7070440938707003E810A828F
:1010400073100134EF00A07F03A74181B7F7FA02C4
:101050009387F70763FDE708370500403706004030
:10106000130505001306560D098E8145EF604015E6
:1010700037460040138541A71306862D098E81450A
:10108000EF600014370600401385818D1306861229
:10109000B7A50080098E93850569EF602014370697
:1010A00000401385819213064627B7A50080098E5C
:1010B0009385056EEF608012138541A7138641A7C3
:1010C000B7B50080098E9385C582EF602011371473
:1010D0000080B7140080EF0080761304041D938411
:1010E000041F6362940E0F00F00FEF500001EF0039
:1010F000407FB7E7003003D707000146136707407A
:101100002390E70003D70701136707402398E70000
:1011100037270028545F9396E6289396F62854DFE5
:101120008356470393E60608231AD7024567130739
:10113000171223AEE70A054798DBD45F985B930547
:10114000C6F98D8A0D8B99C1639DE6063767C10F7D
:10115000B7E7003013077710B8CB23AA07041307AB
:101160002003B8CFB84B1377F7F913670702B8CB52
:10117000B853058B75DFB84BB7D600303706F1FF93
:10118000659B13674700B8CBF8467D16718F131720
:10119000072913171729F8C6F84637E600301367F2
:1011A0002700F8C6094798DB8146585E1C5A93858C
:1011B000C6F90D8B8D8BE38105EAE30FF7E8850611
:1011C000EDB705069DBF1C401104829719BF0000B2
:1011D00036580080525D0080742F0080D832008025
:1011E0002E2C0080DA610080D4620080141600800A
:1011F000C199138705F0996718C19387078823A0C1
:10120000F5F0B7A700809387476523A4F5F0AD6795
:1012100023A2C5F09387A7BB63E3E60082809CC24C
:101220009106DDBF411106C622C4F327003073705A
:101230000430138401C21844A18B050718C473A09D
:101240000730BD2873260030737004301C488507B2
:101250001CC8B70700409387070093858700D843D1
:10126000544391CA5443FD1654C391E65440184761
:101270003397E62858C09107E393B7FE937786002B
:1012800073A007303706000285450CC2F3270030F3
:10129000737004301844A18B7D1718C419C773A04C
:1012A0000730B24022444101828054407D479396EA
:1012B0000660158F144058C4E303D7FE0CC2C5B7AF
:1012C0003747000208434C43B167938707353E9583
:1012D000B337F500BE957D5650C308C34CC382801A
:1012E0002A811243116137470002B7C70002E11794
:1012F000D0438843CC43E39DC5FE4CC308C3C937E4
:10130000056513058588732045300F00F00F736065
:1013100004300283130000001300000013000000DB
:10132000117186DF96DD9ADB9ED9AAD7AED5B2D3EE
:10133000B6D1BACFBECDC2CBC6C9F2C7F6C5FAC3C5
:10134000FEC1732330001ADF02FD06FB0AF90EF717
:1013500012F516F31AF11EEF2AED2EEB32E936E7FD
:101360003AE53EE342E1C6FEF2FCF6FAFAF8FEF692
:10137000F322003079737D1333F36200731003306E
:10138000F32310341EC216C07311013473252034A8
:1013900063580512732540349355B54881C5EF0055
:1013A0006047CDBF9355754881C5EFF0BFE7DDB706
:1013B0009355354863880510732500348322050052
:1013C00020D564D123202507232E3505232C450560
:1013D000232A55052328650523267505232485051D
:1013E000232295052320A505232EB50363D80202E9
:1013F00000FD44F927282503272635032724450324
:101400002722550327206503272E7501272C8501E8
:10141000272A95012728A5012726B501B70500022F
:1014200023A00500EF00001473100534731101347C
:101430008242124373900230731013347A53731044
:1014400033006A70DA704A71BA712A729A720A733A
:10145000FA636A65DA654A66BA662A679A670A684D
:10146000F678667ED67E467FB67F6274D274427905
:10147000B279227A927A027BF26B626CD26C426D04
:10148000B26D265496540659F649664AD64A464BDA
:10149000B64B264C964C064DF25DFE50EE525E5316
:1014A000CE533E55AE551E568E567E47EE475E488D
:1014B000CE483E4EAE4E1E4F8E4F1161730020300F
:1014C000EF00C03773110134F322003063D90202F8
:1014D0007A53731033006A70DA704A71BA712A72E3
:1014E0009A720A73FA636A65DA654A66BA662A67A7
:1014F0009A670A68F678667ED67E467FB67F824215
:1015000012437390023073101334FE50EE525E5348
:10151000CE533E55AE551E568E567E47EE475E481C
:10152000CE483E4EAE4E1E4F8E4F1161730020309E
:10153000010001A05841FD4713170760998F18411A
:101540006301F7025CC50547B707000298C37360E3
:1015500004300F00F00F737004305C451841E3183D
:10156000F7FE8280938701C2944337070040130738
:101570000700B3C6E620944288C2D44733C7E620AA
:1015800018430843D84798C38280B388E5401CCDF0
:10159000B70700402322050093D82840938707000F
:1015A000B347F62010C523260500368618C9232A1E
:1015B0001501BA8688C32DB9411106C622C42A87EF
:1015C0007324003073700430138501C21441B707CF
:1015D000004093870700B3C7F6209C43D8C35C4103
:1015E000B397D7485CC11C4591E3A9372188732084
:1015F0000430B240224441018280AD671449938790
:10160000A7BB01453347D52018436303F700828009
:101610000505CDBF938701C21307000298C31D477C
:10162000D8C323A40700B7970080B716008093871C
:1016300047DE138701A9938626530146938501C28D
:10164000138541A799B72A87138501C254410C43DA
:10165000B3F7D5408DC713960760B7070080B3D79F
:10166000C700DD8E54C1B3F7F5401CC31C4591EB98
:10167000411106C6C135B240054541018280014590
:10168000828005458280011122CC06CE26CA4AC836
:101690004EC62A84F3290030737004305C4199CF20
:1016A00023220500054593F9890073A00930F24013
:1016B0006244D2444249B2490561828003A701C213
:1016C000B704004093840400B34797209C43CCC3E5
:1016D0001C41B397E7281CC1138501C25C41B39735
:1016E000E7485CC183A701C2B3C797209C43C0C72A
:1016F0001C4591E3813503A701C2B3449720944070
:1017000023A606001C4033D6E74801E623A20600C4
:1017100051BFB397E7481CC0014571B7011122CCF6
:1017200006CE26CA4AC84EC62A84F32900307370F2
:10173000043037090040138501C21309090083A74B
:1017400001C25840B317F02809EF5CC093F9890033
:1017500073A00930F2406244D2444249B249056163
:10176000828018405D8F18C05841B377F7405CC144
:1017700083A701C2B3C727219C43C0C71C4581E78B
:10178000553B138501C283A701C2B3C727219C43E0
:1017900023A607006DB7411106C622C4732400308A
:1017A0007370043003A701C2544121883317E02825
:1017B0006388E60073200430B240224441018280F5
:1017C000232205004935FDB719E59387819AB3C5F2
:1017D000F52090C1828093878192D5BFB707000C16
:1017E0003345F5200CC18280B727000C11E59843E2
:1017F0003317B72898C3828003A707083317B72881
:1018000023A0E7088280B707200C19C1B717200C66
:101810008CC38280411122C43704200C26C244406C
:101820009387819AB3C7F4209C4306C699C38297D5
:1018300044C0B240224492444101828001A037E674
:1018400000300328C603344E832806053C4A284A44
:10185000384A2C4A03230605D20693D87800B5836C
:1018600041815983E5811353434813783800D1826D
:1018700093F8F8039D8B1375F5031D8B93F5F50312
:1018800063030300704A130615008507B387C70278
:101890003723F40013030340138615000507B386AE
:1018A0006602B3871703B3D7F6023307C7020946A8
:1018B00033071703B3D6E6023E87630DC8000D4613
:1018C00021676309C8001A876316080037470F00AD
:1018D0001307072423A8F18023A6D18023AAE1803F
:1018E0008280B7E70030B84B799BB8CB23A80704B8
:1018F0008280A98DB7A700809387079893F5F50F8D
:10190000B3A5F52083D7050021813D8D828041114B
:1019100022C426C206C62E84B384C5006317940071
:10192000B240224492444101828083450400050470
:10193000C937EDB703070500838705006396E70005
:1019400091C705058505FDB7014582800545828063
:10195000E546834705001387F7F91377F70F63E52B
:10196000E60081172300F500830715000505F5F350
:101970008280411122C426C22E8406C6AA84EF505A
:10198000300808C00DC12685E137B756002C014745
:101990009305D0037D4585062948B54821431C4061
:1019A0006348F7000545B2402244924441018280D9
:1019B0003386E4008307060063C0F5026349F5003F
:1019C000634EF800635AF3002300060031A081172C
:1019D00033DEF648E31A0EFE0507D1B7E39E17FF84
:1019E000E5B79C4191CB18418306070081EA0507C2
:1019F00018C1FD179CC1F5B701458280054582805D
:101A00009C4199CB18418306070091C6050718C170
:101A1000FD179CC1F5B7F1B70145828083C7818B63
:101A200037670030C5CF93871500B337F000011139
:101A3000B307F04022CC52C433FAF50026CA4AC894
:101A40004EC656C206CEAE842A89138441208149EF
:101A5000938A4182F32700307370043003570400E7
:101A6000A18B2DC30357040021CB035724002297D9
:101A700083466700035704007D172310E4000357D3
:101A8000240005072311E400035624001307000473
:101A90006314E600231104002300D90073A007306B
:101AA000054573A00930F2406244D2444249B2492C
:101AB000224A924A05618280035724003A94834661
:101AC0006400D9BF73A0073081C8D2855685653EB2
:101AD00001C573A00930BDBF0145E1B71C4F93D7C5
:101AE0004748EDFF1C432300F5000545828083072E
:101AF00005001307000C93F7070E639BE70003052F
:101B00001500798D130505F813351500050582803C
:101B100005458280011122CC26CA4AC806CE2A89F0
:101B2000014481446349B400F2406244424926853D
:101B3000D24405618280330589002EC64D3FB245EF
:101B400085042A94C5B783570500130700406387AF
:101B5000E70283574500AA972383B70083574500C0
:101B600085072312F5008357050085072310F5002C
:101B7000835745006394E700231205008280F32712
:101B8000003073700430138701C21447A18B85069F
:101B900014C773A00730B76500309C4D93D74748F2
:101BA000A1E773260030737004309387412013053A
:101BB0000004944D93D64648B5C6F32500307370A3
:101BC0000430544303A541823378D5406318080894
:101BD000938741828546D4C393F7850073A007306D
:101BE0009377860073A00730B76600309C4E93D77A
:101BF000574881EF9387C12403D6070035EA83D77E
:101C0000860393F7F7FD239CF602F32700307370E9
:101C100004301447A18BFD1614C76385061073A00A
:101C20000730828003A8050083D60700E383A6F867
:101C300083D64700BE962383060183D647008506D8
:101C40002392D70083D6070085062390D70083D63A
:101C50004700E390A6F623920700A1BF03284700A0
:101C6000E98E336805012322070123A2D182ADB793
:101C700073260030737004301308004083D50700CA
:101C8000A9C58C4E93D55548A9E183D5070085C9D0
:101C900083D52700BE9503C5650083D50700FD15D4
:101CA0002390B70083D5270085052391B70083D5FE
:101CB0002700639405012391070088C2C1B783D52B
:101CC0002700BE9503C56500CDBF83D7070089EB0C
:101CD000B766003083D7860393F7F7FD239CF6029F
:101CE000F325003073700430544303A5C181337869
:101CF000D540631F08009387C1818546D4C393F7FD
:101D0000850073A007309377860073A00730F5BD78
:101D100003284700E98E336805012322070123AE1B
:101D2000D180F1BF5043FD4613160660918E54C713
:101D30001843E386E6EE37070002854614C3C5B5AF
:101D400083C7818B797126D206D622D44AD04ECE53
:101D500052CC56CA5AC85EC6AA8437670030D5C36B
:101D60001384C124BA89130B00401389C181814AAD
:101D7000732A00307370043083570400A9CB835753
:101D800004000147B307FB40B3C7070891C793F5A9
:101D9000F40F22854D3B0547F32700307370043064
:101DA00023220900A18B73A00730137A8A007320C5
:101DB0000A3029C373A00A30B250225492540259F7
:101DC000F249624AD24A424BB24B4561828083A7B4
:101DD000890193D7574881E723A099006DBF93F5F8
:101DE000F40F22858D3383D7890393E70702239C61
:101DF000F90255B781454A85EFF0FF8873A00A3094
:101E000085BF1C4F93D75748EDFF04C375B75D716D
:101E10004AD052CC2A8A1385C18222D426D24ECEF1
:101E2000BAC0BEC206D62EDA32DC36DEC2C4C6C6A0
:101E3000EFF0DF8E938741202390070003D7270020
:101E4000B744004001442392E700A1499384842DC4
:101E5000FD556800E1360305C100930735FF9DC7B6
:101E6000930765FF85C7E93D8307C100639A370182
:101E700065D013050002E9354E857D14D135C9BF03
:101E8000338784002300F7000504D9B737450040A5
:101E90001305852D50182A94D28532C623000400DC
:101EA000EF5080192A841385C182EFF0DF8EB25083
:101EB0002285225492540259F249624A6161828019
:101EC000B7E700309843411106C622C413670710D4
:101ED00098C3984B3764003037260080136707108B
:101EE00098CB98471306E6B7D9451367070498C7F8
:101EF000984F01451367070498CF37070028545FB0
:101F0000ED9A54DF545F93E6560054DF8D4654DB60
:101F1000145393E6160014D3416713071710B8DB68
:101F2000A1475CD09307C0021CD4930700075CD480
:101F300083474403E19B93E73700230AF402834776
:101F4000440393F777FC93E78701230AF40293078E
:101F500000051CDCEFF05F8785455945EFF01F88D1
:101F6000D9450145EFF05F8893071030B2401CD887
:101F7000224441018280797126D283C7818B22D489
:101F800006D64AD04ECE52CC2A842E8699C71385C7
:101F9000C1822EC6EFF08FF83246A285374400404A
:101FA00013058431EF50400063550504B799008054
:101FB00003C9818B0144238C018A9389C9DE130AEA
:101FC0008002B3073401038507000504953BE31A3B
:101FD00044FF238C218B83C7818BB9CF2254B2500D
:101FE00092540259F249624A1385C18245616FF0E9
:101FF0008FFA9307004063C4A702130484313309A6
:102000008500A949E30924FD83070400639437018F
:1020100035453D330305040005041D33E5B783C78B
:10202000818B89C71385C182EFF0EFF63795008069
:10203000130585E1EF40A003B25022549254025997
:10204000F249624A4561828039712ED24C1006CE27
:1020500032D436D63AD83EDA42DC46DE2EC6213FAE
:10206000F24021618280397122DC2EC62A842E85BD
:102070002C0006DE26DA4AD84ED652D456D25AD092
:1020800032C4EFF01F8F6307051C2C006800EFF0CF
:102090005F956301051C3245B7950080938505E780
:1020A000EFF05F89B7940080630B05168327445CCB
:1020B000B7A50080379500809C47938545C21305DE
:1020C00085E7829732459385C4E7EF502015324566
:1020D0009385C4E7EFF01F86B79500806309051468
:1020E0008327445C37960080379500809C47130611
:1020F00006E8938505EB130585EB829732459385BA
:10210000C4E7EFF03F83B79500806305051683278A
:10211000445C37960080379500809C47130606F292
:10212000938545F5130585EB829732459385C4E782
:10213000EFF05F80B7950080630605168327445C47
:1021400037960080379500809C47130686FB938561
:1021500085FF130585EB829732459385C4E7EFF041
:102160006FFDB7950080630005168327445C3796A2
:102170000080379500809C47130606029385C504AE
:10218000130585EB829732459385C4E7EFF08FFA0C
:10219000B7950080630605148327445C379600805A
:1021A000379500809C47130646059385C510130597
:1021B00085EB829732459385C4E7EFF0AFF7B7958B
:1021C00000806305051E8327445C379600803795A1
:1021D00000809C471306C6149385051B130585EBE9
:1021E000829732459385C4E7EFF0CFF4B79500802E
:1021F000630105288327445C37960080379500806B
:102200009C471306861D93854524130585EB82970D
:102210008327C45C2246B2450325445C05A43245AD
:102220009385C4E7EFF00FF1E31205E84DB53245B1
:10223000938505EBEFF00FF0E30205ECEF10E006FD
:102240008327445CAA859C4705C137950080130508
:1022500045EC8297F2506254D2544259B259225AF4
:10226000925A025B2161828037950080130585EFC9
:102270008297CDB73245938545F5EFF0AFEBE30696
:1022800005EAEF00B07F8327445CAA859C4711C50F
:10229000379500801305C5F56DBF37950080130590
:1022A00005F9F9B73245938585FFEFF0AFE8E3050F
:1022B00005EAEF0070798327445C379500801305A9
:1022C00005009C4775B732459385C504EFF08FE64E
:1022D000E30B05EA8327445C8847EF0070719DBFDC
:1022E00032459385C510EFF0EFE4E30505ECB24706
:1022F000038707009307F003630AF7002C006800C8
:10230000EFF00FF001E58327445CB1AA3245B794A2
:102310000080300893854411EF40903BE247E5D7B9
:10232000B247038707009307F0036307F7002C0009
:102330006800EFF0EFEC61D93245700893854411E5
:10234000EF401039B247038707009307F003630794
:10235000F7002C006800EFF0AFEA55D58327C4538F
:102360006246F24681EF324522476314F702229714
:10237000230207542320D454232EC4528327445CC1
:1023800037950080930544549C4713058511829727
:10239000D1B5B305F5008385050099E193050002E9
:1023A0003308F4002302B8548507C1B7324593853A
:1023B000051BEFF02FD8E30605E2B24703870700BD
:1023C0009307F0036307F7002C006800EFF04FE37A
:1023D0001DD9324A9307F00303070A006307F70089
:1023E0002C006800EFF0CFE119DD324B2249930950
:1023F00044208144B14A83A509005285EFF08FD370
:1024000021CD130640043386C40281473307C4003C
:1024100063C8270393074004B384F402130686209D
:102420003795008022961305851BA29426992304D4
:1024300009208327445383A544209C47829719BDD4
:10244000B306FB008386060099E29306000223048C
:10245000D720850705076DBF850493894904E39C50
:1024600054F9832744539C4737A50080130545C082
:1024700001B5324593854524EFF0CFCBE30A05D86B
:10248000B247038707009307F0036308F7002C00A7
:102490006800EFF0EFD6E30805E6B24AB795008092
:1024A0009385C5245685EFF0EFC8AA891309442007
:1024B0008144314A63830902230209008504130918
:1024C0004904E39944FF832744539C47E38E09F86A
:1024D000379500801305452661BB83250900568585
:1024E000EFF04FC561DD93074004B384F4023795E4
:1024F000008013050525A2942384042083274453D8
:1025000083A544209C47B1B393074004B385F502EB
:10251000B307B5000387470015C33E870145930500
:102520000004830647003308A6002300D80081CAB0
:1025300005050507E317B5FE2382070001458280E4
:102540008327455C5D714EDE9C47AE898325855CA3
:10255000A6C2AA8437950080A2C4CAC052DC56DA4B
:102560005AD85ED686C662D466D26AD0130585E78D
:10257000829701490144ED4A354A130BF007A14BFC
:1025800083A7445CFD551305E101DC438297630892
:10259000055E0305E1016318553D83A7445C93057F
:1025A00040061305E101DC43829779D983A7445C97
:1025B0000307E1019306F004DC436304D734930678
:1025C000B005E31FD7FAFD551305E10182976308B3
:1025D000055A8347E1015D479387F7FC93F7F70FAF
:1025E000E360F7FA37A70080130707B8B3C7E720FF
:1025F0009C438287214C0389140093156900890547
:10260000A6952E852EC6EF40B03FB24521C52A843F
:102610004E85EF40B04083C71400FD179397476085
:1026200063D307009D47A380F40083A7445C3795DC
:102630000080130585279C47829783A7445C83A568
:10264000845C379500809C474E8613050528829749
:1026500022893DB79307F9FF9397476063D307003B
:102660009D477D1CA380F400137CFC0FE3150CF840
:1026700023800900014455BF21491D4483C514002E
:102680008505939545606353B4008145A380B400EC
:102690009A058905A6952E852EC6EF407036B2455F
:1026A00011C52A844E85EF40703741B77D191379E3
:1026B000F90FE31509FC6DBFE35489EC03AC445CEE
:1026C00033852901EFF0AFC283278C002A99379513
:1026D000008013058528829765B5E30309EA05455F
:1026E000635725011305E9FF4E95EFF04FC083A70F
:1026F000445C3309A940379500809C471305C528E1
:10270000D9BFE30F09E683A7445C9C473795008057
:10271000CA8513050529829701499DB583A7445CA5
:10272000FD551305E101DC438297E30B05E4030744
:10273000E101130CE00783A7445C63158701E30103
:1027400009E4E1B7DC43FD551305F1018297E30984
:1027500005E28307F101E39587E38347E101214720
:102760009387F7FC93F7F70FE36CF7E037A7008048
:10277000130707BEB3C7E7209C4382879D454E865B
:102780001385442051332A84E30C05DE83A7445C7F
:1027900083A5845C4E869C47379500801305852968
:1027A0008297B6402285264496440649F259625AD9
:1027B000D25A425BB25B225C925C025D61618280B4
:1027C000954575BF914565BF8D4555BF894545BF49
:1027D000854575B7814565B7994555B783A7445C6D
:1027E000FD551305E101DC438297E30B05D883A770
:1027F000445CFD551305F101DC438297E30205D8E3
:102800000307F1019307E007E31CF7D68307E10113
:10281000130730036384E702634CF70013070003D8
:102820006380E70213071003A545E38AE7F489BB39
:1028300013074003AD45E384E7F499B3A94581B795
:10284000A14535BF83A7445CFD551305E101DC4379
:102850008297630605320307E1019307E007E3115E
:10286000F7D2E35F89D083A7445C37950080B30536
:1028700024419C471305052A8297D9BB83A7445C52
:10288000FD551305E101DC438297630A052E83079A
:10289000E101938727F8E39507CEE35389CE33050B
:1028A00024418547338C29016305F5006285EFF0EB
:1028B0000FA4CA873307F5004E97830607003387B6
:1028C000F90085072300D700E356F4FE83A7445C94
:1028D000098C379500809C47E2851305852A8297ED
:1028E000B30524416285EFF0EFA2AA85E30A05C88B
:1028F00083A7445C37950080130505299C47829780
:1029000041B1FD551305E1018297630A052683074E
:10291000E101130720056385E704634DF700130702
:1029200000056380E70213071005E39BE7C44E86AA
:10293000854511A813073005E394E7C44E868D45FD
:1029400019A04E868145138544207D3EE30A05C2C9
:1029500083A7445C83A5845C4E869C472A842DBD56
:102960004E868945CDB7630E45076340AA046308C8
:10297000750FA9476307F50693270502E39207C081
:102980009327E403E38E07BE631F24171309140083
:102990004E942300A400B38729012380070083A756
:1029A000445C4A849C438297E1BEE31765FDE3598A
:1029B00089BC330524418547338C29016305F50023
:1029C0006285EFF0CF92CA873307F5004E978306F2
:1029D00007003387F90085072300D700E356F4FE8C
:1029E000F5B5B38789002380070083A7445C83A5DE
:1029F000845C379500809C474E8613058529829715
:102A000083870900E38F07D8138A24000149A14A6C
:102A1000D2854E85EFE01FF201C5A380240151B39A
:102A200005091379F90F130A0A04E31359FF038503
:102A30000400CE851A0509052695EF40207E838780
:102A400004001D47A380F400850793974760634502
:102A5000F7002380F400B1B32380040099B3631A14
:102A60002403E30F04B00545635785001305E4FF15
:102A70004E95EFF0CF87098CB3878900238007003C
:102A800083A7445C379500801305052B9C478297EC
:102A9000C1B6E35789AEE30509AE05456357250185
:102AA0001305E9FF4E95EFF08F84CA873387F9004D
:102AB000830607003387A7404E972300D70085077A
:102AC000E356F4FE83A7445CB30CA940330CA44046
:102AD0009C4737950080B38599011305452B829754
:102AE000B305244133859901EFF0CF82AA8509C946
:102AF00083A7445C37950080130505299C4782977E
:102B000066896284B5BCE35D89A61387F9FFB38744
:102B10008900CA854A976315F704B3872901238082
:102B2000A70083A7445C03C78181130C19009C474D
:102B3000130D140019C39305F9FF37950080CE9546
:102B40001305C52B8297B305244133858901238C56
:102B50000180EFE03FFCAA8511E962896A840DB427
:102B600083C60700FD172381D70075B783A7445C90
:102B700037950080130505299C478297F9BF0144CA
:102B80000DB139715AD0138B811B52D45ECE06DE43
:102B900022DC26DA4AD84ED656D2370A0040938B2A
:102BA000811713044A430329C4536306090283C7E8
:102BB000918195CF8149930A0002832784538145EF
:102BC0001305F100DC43829711C98307F100639775
:102BD0005701232E0452A38C01800DA8832704548F
:102BE000638737010545EFE03F9D8509F9B78547C4
:102BF000DE857D195A85A38CF180232E2453EF4066
:102C0000E0615A85EF40C05F2A8611E9B7070040AE
:102C1000DA8513854743EFF0BF922A8659D1B7076B
:102C20000040DA8513854743EFF0EFC39DBF4111A4
:102C300022C406C69387C18223A0070023A20700EF
:102C40009387C12423900700239107002392070054
:102C500093874120239007002391070023920700C8
:102C60009387418223A0070023A207003704004076
:102C70009387C181232A04421304444323A00700FD
:102C80001305442013060033814523A207002320A7
:102C90000404232004082320040C232004102320F0
:102CA0000414232004182320041CEF406051B7971C
:102CB00000809387072C2322F420B7970080938706
:102CC000472C2324F424B79700809387872C23264E
:102CD000F428B79700809387C72C2328F42CB79744
:102CE00000809387072D232AF430B79700809387BD
:102CF000472D232CF434B79700809387872D232EFC
:102D0000F438B79700809387C72D2320F43EB797F8
:102D100000809387072E2322F442B7970080938781
:102D2000472E2324F446B79700809387872E2326C7
:102D3000F44AB79700809387C72E2328F44EB7A78D
:102D4000008093878765232AF452232CF452232290
:102D5000F45CB79700809387072F2324F45CB76750
:102D60000080938767DBB240232E04522320045453
:102D70002326F45C2244410182803387B6008567B4
:102D800063E3E71839714ED626DA9314C50013852C
:102D9000418322DC4AD852D42E8906DE56D25AD03C
:102DA0005ECE62CC328A3684EFE05F97B707008050
:102DB000BE941375F900CA942DC5814793FA04FF98
:102DC000C146B385FA008C413306F10091070CC26D
:102DD000E399D7FE338BA7401379F50F5A86D28536
:102DE0000A95EF40A03FB7D7003023A05701024714
:102DF000D8C3124798C72247D8C7324798CB37075E
:102E0000DEC00907F8C30100010001000100010054
:102E1000B847058B75FFC1044114B38424415A9A05
:102E20004A94370BDEC0814A3D4C37D90030090B3C
:102E3000B30754416366FC089376F400137704FFEC
:102E4000B9CE419826941C4052973EC05C403EC289
:102E50001C443EC45C443EC68147B305F70083C5AD
:102E600005003306F10085072300B600E397D7FE7F
:102E7000B7D7003080C30247D8C3124798C722474C
:102E8000D8C7324798CB3707DEC00907F8C301001F
:102E90000100010001000100B847058B75FF138593
:102EA0004183EFE05F8FF2506254D2544259B259DD
:102EB000225A925A025BF24B624C05452161828094
:102EC000B38B54014146B3055A010A85EF400031E6
:102ED0002320790182472322F90092472324F90015
:102EE000A2472326F900B2472328F90023226905C7
:102EF0000100010001000100010083278904858B86
:102F0000EDFFC10A35B701458280411122C426C2B6
:102F1000AA841385418306C6EFE05F80B7070800E7
:102F2000A69737D70030B2071CC3B707DEC091079A
:102F30007CC3010001000100010001003C47858BBA
:102F4000F5FF13854183EFE01F85B2402244924490
:102F50000545410182801305F00F45BFB2862E86DC
:102F6000AA851305F00F11BDB7F70F80AA9703C507
:102F7000070082809387418323A0070023A20700D4
:102F800082805C45C9CB94438567214763E6D708B7
:102F9000411126C204414AC0416922C406C62A849E
:102FA0007D1918441C40BA975844584763ECF40202
:102FB0001385170002975C441844AA840840DC4734
:102FC0003A95829793978400C98FB3C7070815472E
:102FD0008144630DF902B2402244924402493A8589
:102FE0004101828026850297AA854A85EFE07F907D
:102FF0002A8985047DB75C44084003294400DC47E6
:103000002695269982972300A90085041C44E3E4B1
:10301000F4FE0147C9B705473A8582805C4579715E
:1030200026D206D622D44AD04ECE52CC56CA854499
:10303000DDCB98438567A14463E7E70A2A8481448E
:103040001C4463ECF40A05491C4408403E955C446A
:103050000505DC4782975C441844931485000840BA
:10306000DC473A958297035684004C40C98C4165F1
:103070007D15EFE0DF892317A100B3C40408639531
:10308000A40081446311090689490149054A5C4449
:10309000D84371CF6319090288438144EF309035DA
:1030A0002A895C44984363EBE40618440C4081464B
:1030B000631FD7068356E1002E974A972300D70057
:1030C000A182A300D700DC438297630105125C4410
:1030D000CA85014598479043029741E98D44639D15
:1030E000490363100908B25022540259F249624A56
:1030F000D24A26859254456182805C400840A6975A
:1031000003C907005C442695DC4782976314A90035
:1031100085043DB701490DBF854995BFDC4726852C
:103120008297B30799002380A70085049DBF504074
:103130003696034506003306D9002E962300A600D6
:103140008506BDB733079900DC47834A070026850B
:1031500082976399AA0885045C449843E3E4E4FEFB
:1031600081444A85EF30D028BDBF8144F5B79C47E4
:1031700010444C400840829735D15C4408401844C4
:103180009C4709469305E1003A95829721D98144ED
:1031900029A85C400840A69783CA07005C4426958E
:1031A000DC4782976392AA0485041C44E3E3F4FE9F
:1031B00081441C4408403E955C440505DC478297E9
:1031C0005C441844AA8A0840DC473A958297939752
:1031D0008A000357E100C98FB3C707086314F700DB
:1031E000E38104F09944E5BD9944E1B78944C5BD44
:1031F000411126C29384C1848C4022C437A600802A
:103200002A843795008006C6130686F513054530D7
:10321000029483C5440037A60080379500801306CA
:1032200046F3130545310294A287224483C5540016
:10323000B240924437A6008037950080130606F10D
:103240001305453241018287411122C4138541850E
:1032500006C6EFE0AFCC373756789387C1841307A3
:10326000274198C315671307A75A2392E7001385D0
:1032700041852244B24041016FE0EFD1411122C4A7
:103280001385418506C626C2EFE04FC91385C18369
:10329000CD39AA8413854185EFE0EFCFB2402244B7
:1032A00013F5F40F924441018280411122C4138529
:1032B000418506C626C2EFE06FC61385C183B93BC0
:1032C000AA8413854185EFE00FCDB240224413F567
:1032D000F40F9244410182809387418523A0070027
:1032E00023A207001387C1839387C1845CC3A147CE
:1032F0001CC79387818D94472326070081CAD44732
:1033000091C694435CC714C3A90694C382801387F3
:103310000501AA8783C6050091059107238ED7FE74
:1033200083C6D5FFA38ED7FE83C6E5FF238FD7FEC6
:1033300083C6F5FFA38FD7FEE31EB7FCB7A50080B9
:10334000B7A8008011489385C50793888866130342
:10335000C002137E38008347C5000346D50083466C
:10336000E5000347F50063150E022E96AE962E97E4
:10337000AE97034E060003C606008346070003C748
:10338000070093572800C69783C70700B347FE007E
:10339000034E050005081105B3C7C7012306F50054
:1033A0008347D5FF3D8E8347E5FFA306C500BD8E4D
:1033B0008347F5FF2307D5003D8FA307E500E31AF8
:1033C00068F8828012059388050111432E87814792
:1033D0003308A600B306F800034E070083C60600B4
:1033E00085070507B3C6C601A30FD7FEE39467FEA2
:1033F00091051105E39C15FD828093577500B30775
:10340000F040ED8B06053D8D1375F50F82805971E7
:10341000A2D4D2CC2A842EC22E8637AA0080AA85B6
:103420002945D6CADAC8DEC6E2C486D6A6D2CAD034
:10343000CECEE6C2EAC06EDE254C6937930A440060
:10344000130ACAF7114B930B0401034794008347F7
:10345000D400A289A306E40003475400A286A30473
:10346000E40003471400A300F40083472400A302F0
:10347000E4000347A4002305F4008347640023010C
:10348000E4000347E4002307F400834734002303E8
:10349000E40003477400A301E4000347B400A3035E
:1034A000E4000347F400A307F400A305E400368713
:1034B000814703460700850793F7F70F52960346A7
:1034C00006001107230EC7FEE39567FF8506E3900C
:1034D000DAFE1246A2856285F53563010C1083CDB4
:1034E000090003CD190083CC29006E8539372AD60F
:1034F00029372AD419372AD26A8501372AD0F53DCF
:103500002ACEE53D2ACC6685CD3D83C439002ACA42
:10351000ED352A89DD352AC82685C5352AC6F13D0F
:103520002AC4E13DA255325E925E0256E246B3479E
:10353000BE00B3C7FE004247B18FB58FB347F90055
:10354000B98FA98FB347FD007243B3C7FC00A58FA5
:10355000524F2380F900B3C7CE00B347F30022488F
:10356000B58FB347FF00B98FB347F800A98FB3C732
:10357000FD00B3C5D501B3C7FC00B58D334EDE01E8
:10358000B248A58F334FBF003343C301A380F90076
:10359000B3C66600B347E901B98F358FB3C7F800EA
:1035A000B3C8E80033481801A98F33450501B3C7F4
:1035B000FD00B3CDAD00B347FD00334DBD0133C6B3
:1035C000F400B3CCAC012381C900A3819901910916
:1035D000E3973BF17D1C137CFC0F85BDB650265450
:1035E00096540659F649664AD64A464BB64B264C7F
:1035F000964C064DF25D6561828011BBAE87AA854F
:103600003E8531B503D70500398D931745003D8DB3
:103610001375F50F9317850093163500B58F218329
:10362000B98F1181A98F2390F5008280011122CCDE
:1036300006CE2A8483471400034704002E85A20780
:10364000D98F9305E1002317F1006D3F8357E10007
:10365000F2402300F400A183A300F400624405615A
:103660008280657123286117032B050023248118AC
:10367000232291182320211923261118232E3117D4
:10368000232C4117232A511723267117232481172E
:10369000232291172320A117232EB115B36766218A
:1036A000131736001CC12A842E89B28463F5E70003
:1036B0005C4185075CC1930784063EC0B7A70080C4
:1036C000135B3B0093870721137BFB03130A000462
:1036D000930A8402930901053EC28DEC8320C11830
:1036E0000324811883244118032901188329C11751
:1036F000032A8117832A4117032B0117832BC11635
:10370000032C8116832C4116032D0116832DC11520
:1037100059618280B30B6A41B3DB9B0ACA8533854A
:103720006A015E865E9BEF30702B5E99B3847441B4
:10373000E3154BFBD687180883C63700910711079E
:10374000230ED7FE83C6E7FFA30ED7FE83C6D7FF9F
:10375000230FD7FE83C6C7FFA30FD7FE8246E39D84
:10376000F6FC832E8400032EC400130600040C080C
:103770004E8576C672C4832D0401032D4401832C2B
:103780008401032CC401832B0402032B4402EF3079
:10379000F024B24E224E4E87145F504393D53661CB
:1037A00093D71661AD8FA9820C43B58F545311077F
:1037B000AE96B6979355266193567660AD8E0D8280
:1037C000B18EB6975CDF1C0AE318F7FCEA8FEE8532
:1037D000728876855E83628FDA836686814893027B
:1037E00000101357B66093576660B98F13579661F0
:1037F000B98F1247B386190194424697184391082E
:103800003697BA97B376E6013377C340358FBA97C8
:10381000B3867700135725609357D5603D8F935734
:1038200065613D8FB347B800B373B800E98FB3C784
:103830007700BA97B6973387F6019A83AE8F639C69
:1038400058021A9BBE9E2A9EC29D2E9DBA9C329CF7
:10385000FA9B232264032324D4012326C4012328B2
:10386000B401232AA401232C9401232E84012320B4
:103870007403014B9DB5C2857A832A88328F3E85B9
:103880003A8685B75971A6D20441CECE9309700706
:1038900093D73400A2D4CAD02A842E89B389F940A0
:1038A00013067004930700F881451305910086D62E
:1038B00093F9F9032304F100EF3090109387090581
:1038C0008A9713D78400A38FE7FA13D70401238FB5
:1038D000E7FA5840238097FC138699009356870097
:1038E000238EE7FAA38DD7FAE180935607012C00C7
:1038F00061832285A38E97FA238DD7FAA38CE7FAEA
:103900008D338347B4002300F9008347A400A3004C
:10391000F900834794002301F90083478400A30141
:10392000F9008347F4002302F9008347E400A3026F
:10393000F900B650265496540659F64965618280BE
:10394000011122CC26CA06CE4AC84EC652C483C72D
:1039500025001307E00F03CA3500AE842A84B105A1
:103960006392E710F9572300F500A300450183C7D0
:10397000640019059549230EF5FE83C774000149BB
:10398000A30EF5FE83C78400230FF5FE9C44A1839C
:10399000A30FF5FE03C63400EF30500483C7340094
:1039A00099073E9483D704002300F40083D70400D2
:1039B000A183A300F40063090900354693856411CF
:1039C00013052400EF309001F2406244D2998D0932
:1039D00033053901D2444249B249224A33450508E8
:1039E000056182803A89137AF90F637946011307DA
:1039F000F9FFB386E4008386C600EDD62300F40009
:103A0000A300440183C744004A861305A400230190
:103A1000F40083C754002909A549A301F40083C712
:103A200064002302F40083C77400A302F40083C778
:103A300084002303F4009C44A183A303F40083D7F0
:103A4000A4002304F40083C7B400A304F400EF30FF
:103A5000E0784A9403C9440013791900E30409F497
:103A6000354989B752890546BDBF03463500AE8743
:103A7000238005003336C0009305C5003E856F30B6
:103A8000E0750346350009479305C5003356E60A3D
:103A90001385C18E2396018E6F304074317152D5DB
:103AA0003A8AD84122DD26DB56D306DF4AD94ED7E3
:103AB0005AD15ECF62CD66CB6AC923800500BD476F
:103AC0002A84AE84B68A63EFE702B7A700809387A3
:103AD000C717B347F7209C4382871307D00F894746
:103AE000631EE60ADCC1F557A30105002301F500BA
:103AF00083C70501F99B2388F400FD572300F400D8
:103B0000A300F40003C704008547631EF700834742
:103B10006400A384F40083D7C40099E323970400CE
:103B200085072396F40083473400A381FA00DC4024
:103B30002322FA0083C784002304FA0083C7940079
:103B40008507A304FA0083D7C4002316FA0083C7AD
:103B500024002317FA0083C704012308FA0003C7CF
:103B60000400238104008947631AF7008347541136
:103B700003474411A207D98F2390FA00FA506A54E0
:103B800003C504004A59DA54BA592A5A9A5A0A5BA8
:103B9000FA4B6A4CDA4C4A4D296182801307E00FD8
:103BA000E312E6F6DCC1F957A30105002301F50095
:103BB00083C7050193E717003DBFA301C500238418
:103BC0000500B285EFF09FA683C70401858B99C7D6
:103BD00023020400A3020400954711A08D47DCC016
:103BE00015B72302C5000547637BC70083C72500BF
:103BF00023800500D8C1BA972381F50021B7B2858B
:103C0000EFF0DFA29147E1BFA302C500B285EFF05C
:103C1000FFA1D9B72303C500B285EFF03FA19947B3
:103C20007DBFA303C500B285EFF05FA09D4745BFF0
:103C30002304C500B285EFF07F9FA1474DB7A304D1
:103C4000C50023050500A3050500B285EFF01F9E02
:103C500083C70401858B91C783473400C1CFAD472B
:103C6000BDBFA547ADBF8347A50003479500B285FB
:103C7000A207D98F0347B50042075D8F93178600CF
:103C8000D98FA304E50013D78700C183A305F500EE
:103C90002305E500EFF09F99A94791B78347A50059
:103CA00003479500B285A207D98F0347B5004207A5
:103CB0005D8F93170601D98FA304E50013D7870002
:103CC000C1832305E500A305F500EFF03F9669B732
:103CD00083C78500138717002384E500AA972386EE
:103CE000C700B285EFF09F9403C784008347340078
:103CF000E31AF7E0B147E5B58347A5000347950010
:103D00008346B500A207D98FC20637A50080DD8E95
:103D1000994581471305C51BB1483387F500050751
:103D20000583330817032A980328080063FE060555
:103D30009305F7FFE3E3B7FE31473387E702014915
:103D400081452A9718436384E604228532C6EFF042
:103D5000FF8D834704003246B307F640B337F000C7
:103D6000B507DCC0230AC410E30E09D883C784005A
:103D700003466900E3F8C7D81305C4001D8E8145CA
:103D80003E95EF30E043BDBBBA87E365D8FA3147D3
:103D9000B387E7023309F500834549007DB7B9468B
:103DA00089476309D70083471500B307F640B33747
:103DB000F00085072380F40083474400A30AC41061
:103DC000858B91CFBD4703C70400DCC0B547A388EE
:103DD000F4008947E308F7D22380040025B3DC48C8
:103DE00081CB985B19EF03C7040089476313F72061
:103DF0008547DCC013063012A2855685EF30003EA1
:103E000011B38347A400834694008345B400A207FE
:103E1000D58FC205DD8D2685029779F9E9B783C76D
:103E20001501B307F540A381C71283C71501FD171C
:103E300093F7F70FA388F500E39607CC83A9450114
:103E400063890914B7E7096A938777663ED8B7B7DD
:103E500067BB938757E83EDAB7F76E3C93872737FF
:103E60003EDCB7F74FA59387A7533EDEB7570E51F9
:103E70009387F727BEC0B777059B9387C788BEC2D5
:103E8000B7E7831F9387B79ABEC4B7D7E05B938722
:103E900097D103AB85011306000293850901281011
:103EA000BEC602D402D6EFF0CFFB03463400930522
:103EB000240028102906EFF0CFFA09469305441193
:103EC0002810EFF00FFA1D46930564112810EFF04B
:103ED0004FF90C082810EFF0FF9A19469305D411FA
:103EE0000808EF30A01663130510814701481946F2
:103EF000930574112808834C64113ECC42CEEF30F8
:103F0000E02D63050B0E624CF24B03570B00930739
:103F10002B0001496313E908BD4763E9270DB797F3
:103F20005B00938707D8E29703A6C900B3B6870161
:103F3000DE9663EDC60A6316D60083A6890063E7A2
:103F4000D70A83467400B3672921DA97A381D70083
:103F5000834684000507238197012382D70023101D
:103F6000EB00336929211305590019469305741193
:103F70005A95EF30A02683A7C90063E87701639ABA
:103F8000770183A7890063F6870123A4890123A60B
:103F9000790185472380F400A1BD0346740083C6E0
:103FA0001700631CD6000346840083C627006316EF
:103FB000D60083C6070063879601050933490908BF
:103FC000A50789BFB3652921950581470148194691
:103FD000DA9508103ED042D2EF3040209257E3E20B
:103FE00077F9639577018257E3ED87F703A7090314
:103FF00019E38D4745B78347A40083469400834562
:10400000B400A207D58FC205DD8D2685029775D134
:1040100049B7011122CC26CA37170040B716004015
:1040200037240040B71400402A86938606232AC608
:10403000130707379305848D1385C44406CEEFF02C
:10404000FFA59307E5FF93F7F70F8546324663E137
:10405000F6029307848D03C7270023800700369755
:104060002381E7001307D00F6309E600D4C301459D
:10407000F2406244D2440561828009479384C4447B
:10408000D8C3FD57A38104002390F400CDB731714C
:104090004AD93729004022DD26DB62CD06DF4ED724
:1040A00052D556D35AD15ECF1309898DB684834633
:1040B0000901371400403A8C898A1304042395EAD5
:1040C00083274901814989C783C9070093F91900EA
:1040D000F5572301F4000546B30794000387B700A2
:1040E00019E7FD1493F4F40FFD17E399C4FE294A70
:1040F00039A0F9572301F400B2848149194A0347D2
:10410000A9002304B400A30194009307170023051A
:10411000F90083472400A303A40023023401230EE3
:10412000F1001C44A30204002303E400A30E910049
:10413000A18363800618230FE100A30FA1002300D1
:10414000B102A300F102FD57D28A2314F102130B2E
:10415000C101FD1AB3CA0A0863910A188357810284
:10416000930BC400A68A2317F1005E8B03C50B00D6
:10417000FD1A9305E100B3CA0A08EFF0AFC8850B3A
:10418000E3960AFE9305E1006285EFF0AFC783571F
:10419000E100DA94B71600402380F40003473400AE
:1041A0009386D623369793D687002300D700231013
:1041B000F4006384090E83244901E5C083C7040029
:1041C000858BE1CF83C71400371500401946230BB8
:1041D000F4109844DC440C0813057534034934008A
:1041E0003AC83ECAEF20907F9C44D4441306000294
:1041F00013871700B337F700B697DCC4B7E7096A2F
:10420000938777663ED8B7B767BB938757E83EDAA0
:10421000B7F76E3C938727373EDCB7F74FA59387F8
:10422000A7533EDEB7570E519387F727BEC0B77727
:10423000059B9387C788BEC2B7E7831F9387B79A4A
:10424000BEC4B7D7E05B938797D198C49385040128
:104250002810BEC602D402D6EFF0AFC052866C085A
:104260002810EFF00FC04A86DA852810EFF06FBFF4
:104270000946B3052B012810EFF0AFBEB71500407B
:104280009385653428101D46EFF0AFBDB71500408B
:104290009385D5342810EFF0EFDEFA506A54DA54E3
:1042A0004A59BA592A5A9A5A0A5BFA4B6A4C2961F6
:1042B00082802300E102A301F10213D78740C18766
:1042C000230F3101A30F0100A300A1022301B102BA
:1042D0002302E102A302F102BDB503451B002C102D
:1042E000050BEFF02FB2B5B503D7C18EB71700405D
:1042F000938707232396E70013070004A384E700AE
:1043000089467D472385E700368613070009A38584
:104310000700B5BB83A6818F0111396706CE22CC79
:1043200026CA4AC81307071093870190638BE608D3
:104330007167130707206382E608096713070758A8
:104340006383E60883C4018F90431387018F034979
:104350001700D44303C787003715004032C08A8551
:1043600025461305C52336C22304E1003714004057
:10437000EF20D06613040423A54693074004A3044A
:10438000F400CA85FD472685130780083686230575
:10439000F400A3050400E539A28537140040130595
:1043A00004FFEFF0EFD9AA85130504FF6244F24041
:1043B000D244424905616F10600609472384E70033
:1043C00051B70547E5BF23840700ADBF011106CEF5
:1043D00022CC26CA4AC8B72700281307000498CB66
:1043E00083C4018F9387018F03C9170093870191BD
:1043F0009047D4479843DC433715004032C48A8540
:1044000041461305C5233AC03EC236C637140040A4
:10441000EF20D05C13040423C14693072004A304B7
:10442000F400CA85FD4726851307A00C36862305B0
:10443000F400A3050400A139A28537140040130538
:1044400004FFEFF0EFCFAA85130504FF6244F240AA
:10445000D244424905616F00707C797122D44ECEFE
:104460002A84AE89AA85379500801305453306D680
:1044700026D24AD052CC328936C63A8AEFD0DFBC37
:10448000EF00D0492285EF007076B2451385416573
:10449000EF10802B21C9014493854165630A2401F3
:1044A000B34734218843EF00107B9385416539C1C0
:1044B00037990080938541651305C933EFD0DFB884
:1044C000630E0A008D4513854165EF10E02719C979
:1044D000938541651305C933EFD01FB71305140049
:1044E0001375F50FB250225492540259F249624AA0
:1044F0004561828005045DB7797122D426D22A8471
:10450000AE84AA85379500801305453306D64ECE76
:1045100032C6B6894AD0EFD03FB3EF003040228593
:10452000EF00D06CB24513854165EF10E02111E931
:104530008144B25022540259F24926859254456171
:10454000828037990080938541651305C933EFD088
:10455000BFAF9385416585C42685EF00D06FAA84DF
:10456000E38909FC8D4513854165EF10E01D69D194
:10457000938541651305C933EFD01FAD5DBF22544C
:10458000B25092540259F2493795008013054534D0
:1045900045616F00506CB946814501470543294686
:1045A0007D58B307D50083870700938707FD639382
:1045B00065008607B3C8C702FD1693C51500B3E7AB
:1045C000C70246973E97E39E06FD3365C702133543
:1045D00015008280394801468145854601472943B7
:1045E000FD5EB3070501838707007D18938707FDEC
:1045F000B388D702330EF702B3B7D7023E9EB30794
:104600001601B3B8C7003E86B3076702F295C69598
:1046100033B76602B38666023E97E314D8FD32854F
:104620008280797122D426D24AD052CC06D64ECE80
:1046300056CAAA842E8439497D5A29468146268540
:10464000A285EF20A010B30A2101130505032380E2
:10465000AA00A285268529468146EF10B0487D191B
:10466000AA842E84E31B49FD379500808A851305B3
:104670008534A3070100EFD03F9DB25022549254DD
:104680000259F249624AD24A4561828039714AD858
:104690004ED652D456D206DE22DC26DA2A89A30F61
:1046A0000100B7190040B71A00406312090A81459A
:1046B0001305F101EF10A06111E9F2506254D254D8
:1046C0004259B259225A925A2161828037170040CA
:1046D00037140040B716004013070737130404FFD0
:1046E0009386062349A00967130767F46391E70CD3
:1046F00085476316F516938501873685EFF0EFB68B
:1047000083C70187638597140947638CE712638425
:10471000071483A5418F83A7818FE388B7F8379566
:10472000008013054535EFD03F92EF00103083A78E
:10473000418F1305803E23ACF18EEFC0FFE70547A4
:1047400069A8EFF0EF9FAA852285EF10203D8145F3
:104750001305F101EF0010779386C9101384416DA2
:1047600013874A3539D90346F101B725004037157B
:1047700000409385858D1305C54436C6EFF00FB212
:10478000AA84E30405F2B2460967130747F49C467E
:10479000A183638FE706E368F7F40967130707F45B
:1047A0006382E7020967130737F4638BE702B68574
:1047B0002285E31809F8EFF0AF98AA852285EF006B
:1047C000F045F5B58547631CF5083685EFF06FAB0E
:1047D00083C7C18EE39B07EC0D4723A6E186F1B5A5
:1047E0008547631EF5066C083685EFF00FA88347F2
:1047F000C10181EFB727002813070004D8C711476C
:1048000023A6E18623A201864DB5EFF03FBC71BD22
:1048100085476316F50403C63600A5471385019046
:104820003356F60A9385C60023200500232205008F
:1048300023040500EF20901A03A7018623A2E18636
:10484000ADB5F1679387072023AAF18ED9B5B96773
:1048500093870710D5BF896793870758F5B783A754
:104860004187850723AAF18689B5938601C29C4AB0
:1048700001114AC823A0F18637270028184326CA09
:1048800006CE22CC058B41EF03A7C18501E7984AEC
:1048900023AEE18493870780938777C4998F93062B
:1048A000E07C63E5F60683A6019003A7419093851B
:1048B000018FB71700409387C72383C5150003C531
:1048C000018F3714004094C313040423D8C336C4A3
:1048D00093075004A146A304F4003686FD473AC668
:1048E00071472305F400A3050400EFF04FFAA285F9
:1048F00037140040130504FFEFF08F84AA851305D9
:1049000004FFEF00B031014723AE018483A7018685
:104910003387E74085679387873863F4E70023AEE2
:104920000184F2406244D2444249056182804111CF
:1049300006C6238C0186EF00500F13058038EFC0A8
:10494000BFC71305B002EF00F0270D45EFC0DFC66B
:104950001305B002EF0010270D45EFC0FFC5B240B0
:104960001305B00241016F00F025411106C6C137A1
:104970001305C044EFC05FC437A500801305456729
:10498000EF00D026B2401305803E41016FC0DFC268
:104990005171DAC9E2C5854786D7A2D5A6D3CAD157
:1049A000CECFD2CDD6CBDEC7E6C3EAC16EDF23962B
:1049B000F18E9387018F83C5170003C5018F13897B
:1049C00001C2832C0901B71B0040EFF0FF91B7191A
:1049D000004093850B23138509FFEFE07FF6D96430
:1049E0002A8D0144938404F9938A818683270901DF
:1049F000B387974163E9F40C83270901B387974193
:104A000063E1F40CEA85138509FFEF003021A94525
:104A10005685EF00304B6DD103C58186EFF06FDF17
:104A200061DD13850B231C4579771307070CA183E0
:104A3000BA97B337F000C18F81E7EFF08F8401445C
:104A400003C7C18E8947E313F7FA9387C18E83C7E3
:104A500017008144014A3EC28D472386F18EB71765
:104A600000409387C72302C0938D0B233EC6924715
:104A7000639DF4046312041691472386F18E938795
:104A8000018F83C5170003C5018FEFF0FF85938564
:104A90000B23138509FFEFE0BFEAAA85138509FF01
:104AA000EF00D0172E54BE509E540E59FE496E4A48
:104AB000DE4A4E4BBE4B2E4C9E4C0E4DFA5D6D6148
:104AC0006DB50544B5BF054449B79387C18EA38032
:104AD00097009387018F83C5170003C5018F596D18
:104AE000130D0DF9EFF05F80EE85138509FFEFE000
:104AF0003FE52AC483270901B38797416366FD0612
:104B000083270901B38797416365FD06A245B7175F
:104B10000040138507FFEF007010A94513858186BB
:104B2000EF00503A71DD03C58186EFF08FCE69D971
:104B300003A78D008967938717F421836311F70218
:104B400083CA3D001306100881456810B3DACA0A0B
:104B5000EF200067B24556866810EF202068834733
:104B6000C10AE39997F801C80544850493F4F40F4A
:104B7000FDBD054475BF371700409307C738130DB7
:104B8000C102814A3EC403270D0022456C083ACE7B
:104B900003274D003AD003278D003AD20327CD00DA
:104BA0003AD4EFE0BFA533E7540135EB03A7818E7C
:104BB00068081843029793074500130505803EC017
:104BC000130545807D676378A70237950080BE8511
:104BD00013058537EFD04FC7BE502E549E540E5943
:104BE000FE496E4ADE4A4E4BBE4B2E4C9E4C0E4D3D
:104BF000FA5D6D61828003A7818E014A5843029756
:104C00000146824752856C083386C74003A7818ED0
:104C1000C1473356F60A1847410A029729A082472E
:104C20005286E360FAFE910A93FAFA0F93070002A4
:104C3000410DE39AFAF415BF1D7186CE930700204B
:104C4000A2CCA6CACAC8CEC6D2C4D6C2DAC05EDE5C
:104C500062DC66DA6AD86ED6B7240028B7A5008071
:104C6000371500409CC4938505681305C538EFE0EF
:104C7000DF980123EF0090472D44130900047D14B1
:104C800023A82401130540061374F40FEFC0DF922C
:104C90007DF41305007DEFC03F92B79700809387A6
:104CA000475F3EC4B7970080938747463EC683A7B9
:104CB000C1860D47638BE73A636AF704B5C30547BE
:104CC000638FE734938701C28C4B23A0B18683A7FF
:104CD00041866380073C83A6C1861147639BE63A01
:104CE0009D8D89679387077163F0B73A3795008088
:104CF00013054561EFD04FB5EFF03FC723A60186FE
:104D0000B72700281307000498C761A61147E39B43
:104D1000E7FA0145EFF09F970545EFF03F975DB744
:104D200013054006EFC05F89379D00808546130656
:104D3000401F81451305CD38EFF00FFC8547631800
:104D4000F504B79C008013850C39EFD0EFAF130545
:104D5000803EEFC07F86D129B794008037950080D0
:104D60009385443A13054533EFD00FAE452E138596
:104D7000443AAD2D9305400613854165EF00D01CE4
:104D800009ED13054006EFC03F83452171BFB727EA
:104D900000281307000498CB41BFB79B0080138500
:104DA000CB3393854165EFD02FAA13854165EFF092
:104DB0008FFE01E9379500801305053BEFD0CFA8A2
:104DC000C9B7379500801305C53DEFD0EFA7138510
:104DD0004165EFF03F802A8AAE8AEFF09F84B79951
:104DE000008023A8419123AA5191938401C2938703
:104DF000893F3EC003AC0401B7970080379A00801A
:104E000093870741130A4A403EC2854D82471245A7
:104E100005479306803E09462C083ECC52CEEFF063
:104E2000CFE3631EB50F379500801305C541EFD062
:104E3000AFA1372C0028930C00041305400623264D
:104E40009C01EFC06FF70547B79900803795008048
:104E5000938949343A869306C0122C081305454DB0
:104E60004ECCEFF08FDF0547379500803A869306EA
:104E7000C0122C081305454E4ECCEFF00FDE05474F
:104E8000379500809306C0123A862C08130505500A
:104E90004ECCEFF08FDC03AD0401379A0080B79A57
:104EA0000080379B0080130A4A53938A4A54130B9D
:104EB0004B5623289C019305800C13854165EF0018
:104EC000B008630B0510938541651385CB33EFD094
:104ED000AF97938541655285BD2B630F050E5685AF
:104EE000EFD08F963795008001479306803E0546A8
:104EF0002C081305C5565ACCEFF02FD68547AA8D3E
:104F0000631CF50C379500801305C557EFD0CF9380
:104F10002145EFC06FEA192423A6B18765B38949FB
:104F200063173501379500801305C54309B7B72AC4
:104F30000028130B00041305401F23A86A01EFC0CB
:104F4000AFE7B2473795008005473ECCB797008062
:104F5000938707479306803E4E862C081305C54766
:104F60003ECEEFF08FCF6317B50137950080130564
:104F7000854875BD63173501379500801305854A4F
:104F80007DB523A86A011305401FEFC0EFE29848E2
:104F90009D679387075333078741E3F9E7E6EFF00F
:104FA000DF9C854D130CCD3885461306401F814587
:104FB0006285EFF06FD4631EB50113850C39EFD015
:104FC000AF881305401FEFC02FDF852403AC040119
:104FD0002DBD23A86A01C9BF98489D6793870753D1
:104FE0003307A741E3F7E7EC0547379500803A869A
:104FF0002C08930640061305055A4ECCEFF0EFC57A
:10500000054737950080930640063A862C0813051D
:10501000055B4ECCEFF06FC4EFF03F9531B33795A1
:1050200000801305055CB7440080EFD0EF81114983
:105030009384C43C83A7C18663902703379500807F
:105040001305855DEFD04F80EF003016B72700289D
:1050500013070004D8C7BDB1A6851305401FEF0094
:1050600070530545EFF08FE2F1B72245EFC0DFFD49
:10507000EFF01F92379500801305C560EFC0DFFC8D
:10508000854723A6F1863DB9856793878738E3E98D
:10509000B7C683A7C18699C3EFF02FFD0545EFC0C2
:1050A000AFD1B7450080938545311305803EEF00B1
:1050B000704EF5BE83570500130700406387E70273
:1050C00083574500AA972383B70083574500850778
:1050D0002312F5008357050085072310F500835739
:1050E00045006394E700231205008280B727004043
:1050F00083D507D53795008041111305056406C691
:10510000EFC09FF4B7270040B24083D5879437950E
:1051100000801305056541016FC01FF3411122C4D2
:105120001385C18806C6EFC06FDF377700301C4F8C
:1051300093D747488DCFF32700307370043013871F
:10514000418823220700A18B73A00730B7270040B6
:10515000938787942390070003D727001385C1887E
:105160002244B2402392E70041016FC0CFE21C43CA
:105170007DBFB7E700309843411106C622C41367CC
:10518000071098C3984B3774003037560080136768
:10519000071098CB98471306A653DD4513670708F9
:1051A00098C7984F01451367070898CF370700281D
:1051B000545F93F6F6FB54DF545F93E6060554DF25
:1051C000B14654DB145393E6460014D341671307EA
:1051D0001710F8DBA1475CD09307C0021CD49307DB
:1051E00000075CD483474403E19B93E73700230A1D
:1051F000F4028347440393F777FC93E78701230A7C
:10520000F402930700051CDCEFC00FDC89455D4507
:10521000EFC0CFDCDD450145EFC00FDD9307103057
:10522000B2401CD8224441018280411126C213851C
:10523000C18822C406C637740030EFC02FCE835712
:1052400004030945F99B2318F4028357840393F759
:10525000F7FD231CF402B7270040938707D523905E
:10526000070003D727002392E700EFC0EFB41C4CE0
:1052700093D73748EDFF8347C402BD9B2306F40252
:10528000B7270040938787942390070003D7270010
:105290002392E700F3270030737004301387C1872F
:1052A00023220700A18B73A00730F327003073700F
:1052B00004301387418823220700A18B73A0073095
:1052C0008347C40293E707012306F402B77700304F
:1052D000984F1357474819CF03D707031385C18841
:1052E000136717002398E7022244B2409244410119
:1052F0006FC06FCA9843E9BF797122D426D2372490
:1053000000404AD04ECE56CA5AC806D652CC5EC6C7
:105310002A89130404D5B7790030130B0040938415
:10532000C187732A00307370043083570400B9CBEF
:10533000835704000147B307FB40B3C7070899C769
:105340009375F90F2285EFF0FFD60547F32700305C
:105350007370043023A20400A18B73A00730137A6A
:105360008A0073200A30014A39C773200A30B250CC
:10537000225492540259F249624AD24A424BB24BE9
:105380004561828083A7890193D7574889EB23A081
:10539000290183A78189850723ACF1887DB793759F
:1053A000F90F2285EFF01FD183D7890393E7070216
:1053B000239CF90259BF81452685EFC0CFAC7320ED
:1053C0000A3085B7411122C426C2AA841385C18838
:1053D00006C6EFC0AFB42685EFF01FF21385C18873
:1053E0002244B240924441016FC0EFBA411126C23B
:1053F00022C42A841385C18806C6EFC02FB20305D4
:10540000040009C50504EFF03FEFD5BF2244B240C8
:105410001385C188924441016FC0EFB741114AC062
:1054200022C42A841385C18826C206C6B304B400E8
:10543000EFC0CFAE631B94002244B2409244138568
:10544000C188024941016FC00FB50305040005047E
:10545000EFF09FEAC5B7AA8F014881460146130EB7
:105460002002A94E654F13030008B387CF0083873E
:105470000700938837FF13B7170093B818003365F8
:10548000170109C90145B5C6B69503850500133551
:10549000150082806396C703134818003387D50030
:1054A000030707006317F70485060506E31F66FA7E
:1054B0003795008041111305056606C6EF00303BA5
:1054C000E385D7FF631D0800138707FE938877FFE6
:1054D0001337170093B818003367170179F713874C
:1054E000F7F91377F70FE36BEFFA8117939747609C
:1054F00075B7828003570500AA870DCB0357250097
:105500002A970345670003D707007D172390E7001C
:1055100003D7270005072391E70083D62700130749
:105520000040639BE600239107008280035725001B
:10553000B307E50003C567008280011106CE22CCC7
:1055400026CA4AC84EC652C4F327003073700430CE
:10555000138401C21844A18B050718C473A0073037
:10556000377900308327890193D74748B9E3F3247B
:10557000003073700430B7290040938989948327E1
:10558000890193D74748ADCFF326003073700430BC
:10559000584003A64188B375E640C1E1938741882E
:1055A0000547D8C393F7860073A00730A18873A07E
:1055B0000430377900308327890193D7574891EF1A
:1055C000B7240040938404D583D70400B1EF8357F8
:1055D000890393F7F7FD231CF902F327003073705A
:1055E00004301844A18B7D1718C45DCF73A0073019
:1055F000F2406244D2444249B249224A0561828063
:10560000832509004E8593F5F50FEFF0BFAA83A718
:105610004189850723AAF1889DB74C40718FD18DB0
:105620004CC023A2E188BDBFF32900307370043061
:1056300083D704008DC38327890193D7574881EF0F
:105640002685EFF03FEB2320A90083A781898507FA
:1056500023ACF188F1BF83D7040089EB37770030A2
:105660008357870393F7F7FD231CF702F3260030D7
:1056700073700430584003A6C187B375E64091EDBE
:105680009387C1870547D8C393F7860073A0073077
:1056900093F9890073A0093089B74C40718FD18D7F
:1056A0004CC023AEE186CDB754407D47939606604B
:1056B000158F144058C4E30BD7F237070002854614
:1056C00014C32DB779714AD02E898505B335B00042
:1056D00022D4B305B040372400404ECE52CC56CA37
:1056E00006D626D2AA8AB375B900130484948149D8
:1056F000138A4188F3240030737004308357040008
:10570000A18885C72285EFF0FFDE2380AA0073A061
:105710000430054573A00930B25022549254025906
:10572000F249624AD24A4561828073A00430630B19
:10573000090052852EC6EFB01FF509C573A00930C8
:10574000B2454DBF0145F9B739714AD8138901C235
:105750004ED68329090152D4797A22DC26DA56D230
:105760005AD05ECE62CC66CA6AC806DE2A8BAE8B81
:1057700001448144130C0008B54A930C2002654D86
:10578000130AEABF832509011305F100B385BB4065
:10579000CE95EFF03FF329C58307F1008329090176
:1057A00063925703E5D0F25062544259B259225ADB
:1057B000925A025BF24B624CD24C424D2685D25437
:1057C00021618280639797031344140013871400A8
:1057D000DA942380F400B307EB0023800700BA8437
:1057E00083270901B3873741E3FF77FBE39C84F903
:1057F0005DBF13F7F70F63F9EA0219E8138477FF27
:10580000938607FE1334140093B61600558C15E0EA
:105810009306F7F993F6F60FE36ADDFA011793178B
:105820004760A307F1005DB7B356FA48A1DE79D40B
:1058300071BF014481BF9387C18823A0070023A2C1
:105840000700B7270040938707D5239007002391CF
:10585000070023920700B72700409387879423907F
:10586000070023910700239207009387418823A014
:10587000070023A207009387C18723A0070023A264
:105880000700828083570500130700406387E70203
:1058900083574500AA972383B700835745008507A0
:1058A0002312F5008357050085072310F500835761
:1058B00045006394E700231205008280B72700406B
:1058C00083D507563795008041111305C56806C674
:1058D000EFC08FF7B7270040B24083D587153795C3
:1058E00000801305C56941016FC00FF6B7E70030AE
:1058F0009843411106C622C41367071098C3984BFA
:105900003706000F378400301367071098CB98478D
:10591000E14501451367071098C7984F13670710B3
:1059200098CF37070028545F9396A6499396B649B7
:1059300054DF545FD18E54DF8D6654DB14533766C9
:105940000080130646B49396C62814D34167130704
:105950001710B8DFA1475CD09307C0021CD493078F
:1059600000075CD483474403E19B93E73700230A95
:10597000F4028347440393F777FC93E78701230AF4
:10598000F402930700051CDCEFB01FE48945614574
:10599000EFB0DFE4E1450145EFB01FE593071030BC
:1059A000B2401CD8224441018280411122C406C663
:1059B0003784003083578403094593F7F7FD231C90
:1059C000F402B7270040938707562390070003D7B8
:1059D00027002392E700EFB03FBE1C4C93D7374817
:1059E000EDFF8347C402BD9B2306F402B7270040A6
:1059F000938787152390070003D727002392E7009A
:105A0000F3270030737004301387C1892322070005
:105A1000A18B73A00730F327003073700430138715
:105A2000418A23220700A18B73A007308347C40259
:105A30003787003093E707012306F4021C4F93D702
:105A4000474889C7B2402244410182801C43FDB7C8
:105A5000797122D426D2372400404AD04ECE56CA7D
:105A60005AC806D652CC5EC62A8913040456B78992
:105A70000030130B00409384C189732A0030737087
:105A8000043083570400B9CB835704000147B307A0
:105A9000FB40B3C7070899C79375F90F2285EFF04C
:105AA0007FDE0547F32700307370043023A2040023
:105AB000A18B73A00730137A8A0073200A30014A41
:105AC00039C773200A30B250225492540259F24915
:105AD000624AD24A424BB24B4561828083A7890118
:105AE00093D7574889EB23A0290183A7018B85070A
:105AF00023A8F18A7DB79375F90F2285EFF09FD81F
:105B000083D7890393E70702239CF90259BF814594
:105B10002685EFB05FB773200A3085B7411122C4E4
:105B200026C206C62A84B304B50063179400B240A7
:105B30002244924441018280030504000504EFF0F1
:105B40003FF1E5B7011106CE22CC26CA4AC84EC69F
:105B500052C4F327003073700430138401C2184418
:105B6000A18B050718C473A007303789003083273D
:105B7000890193D74748B9E3F324003073700430A8
:105B8000B7290040938989158327890193D747480E
:105B9000ADCFF326003073700430584003A6418A1D
:105BA000B375E640C1E19387418A0547D8C393F7AF
:105BB000860073A00730A18873A0043037890030B5
:105BC0008327890193D7574891EFB72400409384E6
:105BD000045683D70400B1EF8357890393F7F7FD89
:105BE000231CF902F3270030737004301844A18B92
:105BF0007D1718C45DCF73A00730F2406244D244D1
:105C00004249B249224A05618280832509004E85B6
:105C100093F5F50FEFF01FC783A7C18A850723A669
:105C2000F18A9DB74C40718FD18D4CC023A2E18A7F
:105C3000BDBFF32900307370043083D704008DC3D7
:105C40008327890193D7574881EF2685EFF09F8AF4
:105C50002320A90083A7018B850723A8F18AF1BF20
:105C600083D7040089EB378700308357870393F786
:105C7000F7FD231CF702F326003073700430584000
:105C800003A6C189B375E64091ED9387C1890547A5
:105C9000D8C393F7860073A0073093F9890073A0E7
:105CA000093089B74C40718FD18D4CC023AEE1884B
:105CB000CDB754407D4793960660158F144058C465
:105CC000E30BD7F237070002854614C32DB779716D
:105CD0004AD02E898505B335B00022D4B305B04033
:105CE000372400404ECE52CC56CA06D626D2AA8AB7
:105CF000B375B900130484158149138A418AF324CA
:105D000000307370043083570400A18885C7228552
:105D1000EFF04FFE2380AA0073A00430054573A066
:105D20000930B250225492540259F249624AD24A7E
:105D30004561828073A00430630B090052852EC632
:105D4000EFB07F9409C573A00930B2454DBF01453E
:105D5000F9B7B72700409387075623900700239190
:105D6000070023920700B7270040938787152390E9
:105D7000070023910700239207009387418A23A0FD
:105D8000070023A207009387C18923A0070023A24D
:105D900007008280938701C2944B83A7418B89E7D8
:105DA000B307D50023AAF18A63F6D700369523AA54
:105DB000A18A82858280797126D2B794008022D40C
:105DC0002EC62A842E859385C4E706D632C4EFB04A
:105DD0007FB6B795008039CD1C4437960080379543
:105DE00000801306866B9385856C130585EB82977F
:105DF00032459385C4E7EFB0FFB3B7950080630FDA
:105E0000050E1C4437960080379500801306C66E39
:105E10009385C56F130585EB8297B247038707000B
:105E20009307F0036302F72037A500801C44130595
:105E3000453505A832459385856CEFB0BFAF4DD988
:105E4000B247038707009307F003630EF7002C00A7
:105E50006800EFB0FFBA01E91C4437A500801305C4
:105E600045338297D1A232459385C4E7EFB09FAC0A
:105E7000B79500800DC51C4437A600801306063177
:105E80009385C56C37950080130585EB8297B247E3
:105E9000038707009307F003E310F7FC71A2324574
:105EA0009385C56CEFB01FA97DD12C006800EFB0C1
:105EB0003FB5B79400800DC13245700893854411F9
:105EC000EF100001F2453795008023A6B1841C44F1
:105ED0001305C56D829789AA1C4437950080130568
:105EE000456D82975C446C081385441182971C446D
:105EF00037950080130585608297E9B73245938511
:105F0000C56FEFB03FA3E30A05F0B2470387070070
:105F10009307F0036307F7002C006800EFB05FAE53
:105F200005DD32459385C4E7EFB0DFA0B79500806B
:105F30003DC11C44379600803795008013060670DB
:105F40009385C571130585EB829732459385C4E728
:105F5000EFB05F9EB79500806302050E1C44379634
:105F60000080379500801306467B9385857C13055A
:105F700085EB829732459385C4E7EFB0BF9BB79519
:105F80000080630D050C379600801C441306C62A5A
:105F90009385C57EC5BD32459385C571EFB09F9988
:105FA0004DD583A5C1861C443795008013054572E5
:105FB0008297B72700289C431844858BBDEBB79583
:105FC00000809385056B3795008013050573029754
:105FD00083A581891C44379500801305C57382977A
:105FE00083A541891C443795008013050575829768
:105FF00083A5018B1C443795008013054576829755
:1060000083A5C18A1C44379500801305C577829704
:1060100083A541871C4437950080130545798297F5
:10602000EFF0DF89EFF08F8CB2502254925445612B
:106030008280B79500809385C56A71B73245938594
:10604000857CEFB03F8F1DD5B795008037950080D8
:106050001C449385057D1305C57DADBD32459385F3
:10606000C57EEFB03F8DE30405E2152275BFAA851A
:106070007370043037950080238C018A1305457FA7
:10608000372400289304000489C92EC6EFB0DFFB33
:10609000B245B79700801385477F83A74181930658
:1060A00080021307400633D7E702B3D7D7028D46E5
:1060B00044C4010001466312E6020100014644C4E3
:1060C0006310E602FD16EDF602CE7247E37EF7FAA4
:1060D0000100724705073ACECDBF01000506E1BFBA
:1060E00001000506F1BF411106C6EFE0FFB4F5BFA0
:1060F000411106C6EFC0FFA8F5BF411106C6B7E7BC
:10610000003003D7070081450145136707402390FE
:10611000E70003D70701136707402398E700B72775
:10612000002813070020D8C713070004D8C7130797
:106130000024D8D7EFB02FEDEFB09FD883A54181D1
:10614000B7470F009387072433F6F50237A5008081
:1061500013054581B3D5F502EFB01FEFEFD00F92D5
:1061600009C9EFD06F8E37A5008013054583EFB0C6
:10617000BFED0547238CE18A094723A0E1C2B70799
:106180000040938707009C478843EFB06F9537A581
:10619000008041111305458706C6EFB0FFEA373589
:1061A000004013054518EFB04FC59315250037A5DE
:1061B00000801305C58DEFB03FE93735004013056A
:1061C0008596EFB08FC3B2409315250037A50080A8
:1061D0001305C58E41016FB03FE737370040B76602
:1061E0000080B74500403735004041118147130713
:1061F000071A9386660E09469385051A13054518F6
:1062000006C6EFB08FB8B24037370040B76600809F
:10621000B7350040373500408147130747989386CC
:10622000060F0546938545181305859641016FB005
:10623000CFB501A005458280594723A8E18C7D5543
:106240008280411122C483C7818B4AC006C626C200
:106250002A8989C71385C18BEFB04FCC83A40192E3
:10626000F3260030737004300F00F00FF327003472
:106270000A86A18A73A0063003A50192B3F7C70A64
:10628000938707F84A9563FDA70283C7818B89C767
:106290001385C18BEFB02FD037A500801305C58FB4
:1062A000EFB09FDA314723A8E18CFD54814773A0FA
:1062B0000730B2402244024926859244410182803F
:1062C00083C7818B23A0A192F5D31385C18BEFB037
:1062D0008FCCE9BF9387C18B23A0070023A20700BF
:1062E00082800000130806009307050093880500CC
:1062F000639C060C63FAC522370701006368E63623
:1063000037070001130380016374E60013030001E3
:10631000B356660017470000130707063307D70078
:10632000034707009306000233076700630ED70098
:10633000B386E640B398D5003357E5003318D6004E
:10634000B317D500B36817011356080133D5C80237
:106350009316080193D6060113D70701B3F8C802B4
:10636000B385A6029398080133671701637CB700D1
:10637000B308E8001387080063F4B80063F4083931
:106380001305F5FF3307B740B355C70293970701CD
:1063900093D707013377C702B386B60213170701F5
:1063A000B3E7E70063FAD700B307F80063F4D70058
:1063B00063F607359385F5FF131505013365B500C1
:1063C000930500006780000063F8D5009305000086
:1063D0001305000067800000B707010063E6F62A96
:1063E000370700019307800163F4E600930700017B
:1063F00033D8F60017470000130707F833070701E3
:1064000003470700130800023307F7006306072954
:106410003308E840B358E600B3960601B3E8D80065
:1064200033D3E50093DE0801B357D303139E08016D
:10643000B3950501135E0E013357E5003367B700CE
:1064400093560701331606013373D303B305FE02D7
:1064500013130301B3E6660063FCB6003383D80070
:10646000930603006374B300637C132D9387F7FFD7
:10647000B386B64033D3D60313170701135707016A
:10648000B3F6D603B3056E02939606013367D700C1
:10649000637CB700B386E8001387060063F4B60098
:1064A00063F416291303F3FF93970701B3E667001C
:1064B0003307B740931706019315030193D70701DC
:1064C00093D5050113D3060113560601330EF302CB
:1064D000B388F502B385C50293D70801B385C5011A
:1064E000B387B7003303C30263F6C7013706010061
:1064F0003303C30013D60701330666006360C70287
:106500009398080193D80801939707013315050163
:10651000B3871701637EF51E631CC71E1385F6FF44
:106520009305000067800000630A06143707010026
:10653000637CE6189338061093B8180093983800D7
:10654000B356160117470000130707E33307D700B8
:10655000034707009306000233071701630AD714A5
:10656000B387E6403318F60033D3E50093580801AB
:10657000335E130313160801B395F5001356060195
:106580003357E5003367B70093560701B317F5009B
:1065900033731303B305C60313130301B3E6660095
:1065A00063FCB6003305D800930605006374B5009C
:1065B00063760517130EFEFFB386B64033D5160378
:1065C0001317070113570701B3F616033303A60287
:1065D000939606013367D700637C6700B306E80033
:1065E0001387060063F4660063F606151305F5FFCE
:1065F00093150E01B3E5A500330767403355170324
:1066000093D60701337717033303C5021317070126
:1066100033E7E600637C6700B306E80013870600F3
:1066200063F4660063F6060D1305F5FF3307674054
:10663000B35617039397070193D7070133771703CF
:106640003386C60213170701B3E7E70063FAC700F2
:10665000B307F80063F4C70063F807099386F6FFF1
:10666000131505013365D50067800000133306104C
:1066700013331300131333006FF09FC99306000008
:10668000930800006FF01FEC93B7061093B7170044
:10669000939737006FF0DFD53336C500B3B6B60039
:1066A0001336160033E5C60093050000678000002E
:1066B0003387C54093580601131606011356060189
:1066C000930510006FF09FF3370700016378E60031
:1066D00093560601930800016FF0DFE6935686019A
:1066E000930880016FF01FE69386E6FF6FF05FF777
:1066F0001305E5FF338706016FF05FF39385E5FF30
:106700006FF09FCB1305E5FF338708016FF09FC73C
:10671000138506009305000067800000130EEEFF4E
:10672000B30605016FF05FE91303E3FF338716013A
:106730006FF09FD71305E5FF338706016FF05FEB1E
:106740009387E7FFB30613016FF09FD2130806008B
:10675000930805001383050013870500639A060E4E
:1067600063FEC526B70701006364F63EB707000164
:10677000930680016374F600930600013353D6003C
:1067800097470000938747BFB387670083C7070019
:1067900013030002B387D700B306F340638C67008E
:1067A0003397D500B357F50033E7E7003318D60029
:1067B000B318D500935508013356B70213130801D7
:1067C0001353030193D708013377B70233066602E8
:1067D00013170701B3E7E70063F2C702B307F80036
:1067E00033B5070133B7C700133515003377A7005A
:1067F0003307E04033770701B307F700B387C7409B
:1068000033D7B7021395080113550501B3F7B70243
:1068100033076702939707013365F5006372E5025A
:106820003305A80033360501B337E50013361600EB
:10683000B3F7C700B307F040B3F707013385A700EC
:106840003305E5403355D50093050000678000000F
:10685000130E050063F4D50067800000B707010040
:1068600063E6F630370700019307800163F4E60022
:106870009307000133D8F600174700001307C7AF8E
:10688000330707018348070013080002B388F800A4
:106890006386082F33081841B39606013353160157
:1068A0003363D300B3DE1501935F0301B3D7FE0357
:1068B000131F0301B3950501135F0F01B3561501B3
:1068C000B3E6B60013D7060133160601331E0501E1
:1068D000B3FEFE03B305FF02939E0E013367D7019B
:1068E000637CB7003305E300130705006374B5004C
:1068F000637A652E9387F7FF3307B7403355F70365
:106900009396060193D606013377F703B305AF02DA
:106910001317070133E7E600637CB700B306E30013
:106920001387060063F4B60063F8662A1305F5FFC3
:1069300093970701B3E7A7003307B7409316060103
:106940009315050193D5050193D6060193D7070149
:10695000935E0601338FD702B386D502B385D50384
:1069600013D50601B385E5013305B500B387D70319
:106970006376E501B7050100B387B70093550501BC
:106980009396060193D6060113150501B387F5000A
:106990003305D5006368F700B305F7406310F702CD
:1069A000637EAE003306C5403335C5003305650050
:1069B000B387A740B305F740130506003305AE4083
:1069C000333EAE00B385C541B3981501335505017B
:1069D000B3D5050133E5A8006780000063020618FF
:1069E000B70701006370F61C133706101337170042
:1069F00013173700B356E600974700009387C797F1
:106A0000B387D70083C7070013030002B387E700EB
:106A1000B306F340638E67163318D60033DEF500F5
:106A200013530801B35E6E0213160801B395D50027
:106A30003357F500135606013367B7009357070124
:106A4000B318D500337E6E02B385CE02131E0E013D
:106A5000B3E7C70163F2B702B307F80033BE07011B
:106A600033B5B700133E1E003375C5013305A04092
:106A700033750501B307F500B387B740B3D5670297
:106A80001317070113570701B3F76702B385C50250
:106A9000939707013367F7006372B7023307E80083
:106AA00033350701B337B70013351500B3F7A70027
:106AB000B307F040B3F707013387E7003307B74068
:106AC000B355670293D7080133776702B385C502D0
:106AD00013170701B3E7E70063F2B702B307F80043
:106AE00033B5070133B7B700133515003377A70067
:106AF0003307E04033770701B307F700B387B740A8
:106B000033D767029398080193D8080133F56702D9
:106B1000B307C7021315050133E5A8006372F50238
:106B20003305A800333605013337F5001336160058
:106B30003377C7003307E040337707013305A700F9
:106B40003305F5403355D5009305000067800000FC
:106B50009336061093B61600939636006FF01FC258
:106B600093060000130700006FF01FE993B70610AB
:106B700093B71700939737006FF0DFCF63E4B60445
:106B80006372C50413050E009305030067800000BF
:106B90003387C54013530601131606011356060129
:106BA0006FF01FF2B70700016378F60093560601F5
:106BB000130700016FF05FE493568601130780010D
:106BC0006FF09FE3330EC5403333C501B386D54024
:106BD000338366406FF01FFB1305E5FF33876600C4
:106BE0006FF01FD59387E7FF330765006FF0DFD0A5
:106BF0006F0080006F0080006F008007130101FFAD
:106C000023248100232611001304050063140500CA
:106C10001304100013050400EF00C004630A05000C
:106C20008320C1000324810013010101678000005B
:106C3000EF00400163140500EF004001E70005008C
:106C40006FF05FFD03A5418C67800000130101FF19
:106C50001305600023261100EF00C04C130510003F
:106C6000EFF02FDD9305050003A541926F00400969
:106C70009305050003A541926F00005C83A7818CFA
:106C8000130101FF23248100232021012326110069
:106C9000232291001309050013840500639807005F
:106CA00093050000EF00404D23A4A18C9305040040
:106CB00013050900EF00404C9304F0FF63129502A6
:106CC0001304F0FF8320C100130504000324810096
:106CD00083244100032901001301010167800000A2
:106CE000130435001374C4FFE30E85FCB305A44000
:106CF00013050900EF004048E31695FC6FF05FFCB8
:106D0000130101FE232A91009384350093F4C4FFFC
:106D1000232E1100232C8100232821012326310159
:106D200023244101938484009307C00063F4F4009A
:106D30009384070063C4040063F8B4029307C0009F
:106D40002320F500130500008320C10103248101E5
:106D500083244101032901018329C100032A810001
:106D60001301010267800000130905009389C18C9B
:106D7000EF00001583A709001384070063100408BF
:106D80009385040013050900EFF05FEF9307F0FF10
:106D9000130405006312F51203A40900930704000D
:106DA0006392070E63000410032A04009305000099
:106DB00013050900330A4401EF00003C6314AA0ED6
:106DC0008327040013050900B384F440938504006D
:106DD000EFF0DFEA9307F0FF6306F50C832704006A
:106DE000B38797002320F40083A7090003A7470077
:106DF0006310070A23A6018C6F004003832604005A
:106E0000B386964063CA06061307B000637AD704B8
:106E100023209400330794006390870423A0E900A3
:106E2000832744002320D7002322F70013050900FD
:106E3000EF0080091305B40093074400137585FF24
:106E40003307F540E302F5F03304E400B387A740CD
:106E50002320F4006FF05FEF23A2E7006FF05FFCE8
:106E6000032744006396870023A0E9006FF01FFC0E
:106E700023A2E7006FF09FFB930704000324440064
:106E80006FF0DFEF1384070083A747006FF05FF117
:106E90001387070083A74700E39C87FE2322070090
:106EA0006FF0DFF89307C0002320F90013050900F5
:106EB000EF0080016FF01FE9232095006FF01FF7AE
:106EC0001385418D6F00402F1385418D6F00002F7A
:106ED000130101F52322F10A93074020232611080C
:106EE0002326B100232CC108232ED1082320E10A38
:106EF0002324010B2326110B2312F102232E01065A
:106F0000232CA1002324A102EF00802F232EA10017
:106F10002326A1020326C10003A541929707000082
:106F200093878703232EF102930681099307F0FFCD
:106F30009305810123260104232001062313F10276
:106F4000232AD100EF0010248320C1081301010B74
:106F5000678000001305000067800000B70700800D
:106F6000130101F89387F7FF232EF1002328F10086
:106F7000B707FFFF2324B100232CB100938787209C
:106F800093058100232E1106232AF10023260106F2
:106F9000EF00405183278100238007008320C10731
:106FA00013010108678000009306060013860500A0
:106FB0009305050003A541926FF05FFA130101F7F5
:106FC000232481089307402013040500138505003E
:106FD000232611082326C1002324D1002312F10205
:106FE000232CB1002324B102232E0106EF004021FF
:106FF000832681000326C100970700009387C7F509
:10700000232EA1002326A102232EF1029305810144
:107010009307F0FF13050400232601042320010633
:107020002313F102EF0010168320C1080324810806
:10703000130101096780000093060600138605000E
:107040009305050003A541926FF05FF71307000059
:107050006316E6001305000067800000B307E50033
:1070600013071700B386E50083C7070083C6F6FF42
:10707000E380D7FE3385D740678000009307F00197
:1070800063FAB700930760012320F5001305F0FFB2
:10709000678000008327C503130101FE232C8100B4
:1070A000232E11001386050013040500638A0700D0
:1070B00013972500B387E70003A7070063160702AD
:1070C000130504002326C100EF00C00A9305050044
:1070D00013050400032481010326C1008320C1019C
:1070E000130101026F00C004130510006308A7021A
:1070F0009306F0FF631ED700930760012320F4007E
:107100008320C10103248101130101026780000073
:1071100023A0070013850500E70007001305000002
:107120006FF01FFE9305050003A541926FF01FF558
:10713000130101FF232481001304050013850500BA
:107140009305060023A8018C23261100EFF0CF8EB3
:107150009307F0FF6318F50083A7018D6384070090
:107160002320F4008320C1000324810013010101C6
:10717000678000006FF00F8C130101FF2324810052
:10718000130405001385050023A8018C2326110094
:10719000EFF02F8B9307F0FF6318F50083A7018DA5
:1071A000638407002320F4008320C10003248100AE
:1071B0001301010167800000678000006780000004
:1071C00013030500630A06002300B3001306F6FF4D
:1071D00013031300E31A06FE678000001303050083
:1071E000630E060083830500230073001306F6FF79
:1071F0001303130093851500E31606FE6780000055
:107200009307050003C7070093871700E31C07FED9
:107210003385A7401305F5FF67800000930705003D
:1072200003C705009387170093851500A38FE7FE1A
:10723000E31807FE67800000638A050E83A7C5FF79
:10724000130101FE232C8100232E11001384C5FF9E
:1072500063D407003304F4002326A100EFF05FC6D7
:1072600083A7C18C0325C100639E0700232204006D
:1072700023A6818C032481018320C1011301010213
:107280006FF09FC46374F402832604003307D400B4
:10729000639AE70003A7070083A747003307D700D7
:1072A0002320E4002322F4006FF09FFC13870700E3
:1072B00083A7470063840700E37AF4FE8326070070
:1072C0003306D7006318860203260400B386C6007F
:1072D0002320D7003306D700E39EC7F803A6070094
:1072E00083A74700B306D6002320D7002322F70048
:1072F0006FF05FF86378C4009307C0002320F500A7
:107300006FF05FF703260400B306C400639AD7004A
:1073100083A6070083A74700B386C6002320D400B6
:107320002322F400232287006FF0DFF4678000003F
:10733000130101FE2328210103A98500232C8100CC
:107340002326310123206101232E1100232A9100DD
:10735000232441012322510113840500130B06004D
:107360009389060063EC26138397C5001307090071
:1073700093F60748638C0608832444011307300002
:1073800083A50501B384E40213072000032A040047
:10739000930A0500330ABA40B3C4E4021387190004
:1073A000330747011386040063F6E40093040700E3
:1073B0001306070093F707406386070A9305060044
:1073C00013850A00EFF0DF9313090500630A050A2D
:1073D0008325040113060A00EFF05FE08357C40021
:1073E00093F7F7B793E707082316F400232824013F
:1073F000232A940033094901B38444412320240102
:1074000023249400138909001387090093090700B6
:10741000032504001386090093050B00EF10005CA0
:107420008327840013050000B38727412324F40039
:1074300083270400B38737012320F4008320C10190
:107440000324810183244101032901018329C1000F
:10745000032A8100832A4100032B0100130101024A
:107460006780000013850A00EF10005B1309050018
:10747000E31E05F68325040113850A00EFF0DFDB28
:107480009307C00023A0FA008357C4001305F0FF40
:1074900093E707042316F4006FF05FFA13890600E0
:1074A0006FF01FF783D7C500130101F52322910A5E
:1074B000232481092326110A2324810A2320210B56
:1074C000232E3109232C4109232A5109232861093C
:1074D0002326710993F70708130C05009384050010
:1074E000638A070683A705016396070693050004D0
:1074F0002326D1002324C100EFF09F8023A0A40005
:1075000023A8A400032681008326C100631005047C
:107510009307C0002320FC001305F0FF8320C10A5D
:107520000324810A8324410A0329010A8329C1090A
:10753000032A8109832A4109032B0109832BC108EE
:10754000032C81081301010B6780000093070004DE
:1075500023AAF40093070002A30CF102930700038F
:10756000232A0102230DF102232ED1009309F0FFFB
:10757000972A0000938A4A3B130B1000130AA000BD
:107580001304060083470400B33BF0009387B7FD64
:10759000B337F000B3FBFB0063920B0CB306C4409F
:1075A0006304C4029385040013050C002324D10056
:1075B000EFF01FD863003525832741038326810020
:1075C000B387D700232AF10283470400638407228C
:1075D0001304140023200102232601022322310375
:1075E00023240102A3010106232C01068345040084
:1075F000130650001725000013050533EF10C03B9C
:107600008327010293061400631E050413F7070184
:107610006306070013070002A301E10613F78700C2
:10762000630607001307B002A301E1060346040046
:107630001307A0026304E6048327C1029306000037
:107640001306900003470400130707FD637EE60856
:10765000638406042326F1026F000004130414005F
:107660006FF05FF2330555413315AB003365F5001C
:107670002320A102138406006FF05FF70327C101E6
:107680001306470003270700232EC10063440704A5
:107690002326E10213840600034704009307E00257
:1076A000631EF706034714009307A0026318F7044C
:1076B0008327C101130424001387470083A7070011
:1076C000232EE10063D407009307F0FF2322F10289
:1076D0006F00C0043307E04093E727002326E10250
:1076E0002320F1026FF01FFBB3874703130414003C
:1076F00093061000B387E7006FF0DFF41304140063
:107700002322010293070000930690000347040020
:10771000130707FD63FAE608E39A0BFA83450400B2
:10772000130630001725000013058520EF10C02830
:1077300063040502972700009387871F3305F540F0
:1077400083270102130700043317A700B3E7E700FC
:10775000130414002320F102834504001306600083
:10776000172500001305051D230CB102EF10C024DE
:10777000630C050893070000639A070403270102BE
:107780008327C10113770710630A07029387470015
:10779000232EF1008327410313061400B38727012A
:1077A000232AF1026FF0DFDDB387470313041400CF
:1077B000930B1000B387E7006FF05FF593877700B6
:1077C00093F787FF938787006FF09FFC1307C10132
:1077D00097060000938606B61386040093050102FF
:1077E00013050C0097000000E700000013090500D6
:1077F000E31235FB83D7C40093F70704E39E07D059
:10780000032541036FF09FD11307C10197060000C4
:10781000938646B2138604009305010213050C00FB
:10782000EF00C0776FF09FFC130101FE232E1100C3
:10783000232C8100232A91009307F0FF6390F50227
:107840009304F0FF8320C101032481011385040008
:107850008324410113010102678000008357C600A1
:107860000327460093F4F50F93F7F7FD2316F60070
:107870008327460363840704832786031384050054
:107880006352F702832706001387F7FF2320E600E1
:10789000A38F87FE83274600938717002322F600D5
:1078A0006FF05FFA930506002326C100EF10400435
:1078B0000326C100E30805FC6FF09FF8832606014C
:1078C000832706006382060263F0F60283C6F7FF91
:1078D000639C96009387F7FF130717002320F60099
:1078E0002322E6006FF01FF6232EF60293074604CC
:1078F000232AF60293073000232CF602930766042E
:107900002320F6002320E6042303B6049307100087
:107910006FF0DFF8130101FF2324810013840500B9
:1079200083A5450323261100638E050293074404B3
:107930006384F500EFF05F9083270404232A040298
:107940002322F400638007028327C4031305000089
:107950002320F4008320C1000324810013010101CE
:107960006780000083270401232204001305F0FF31
:107970002320F4008357C40093E707022316F40082
:107980006FF05FFD130101D497070000938707EAAA
:107990002326312B2324F1289309C10097070000E7
:1079A000938787F7232C812A2328212B2324412BFB
:1079B000232E7129232E112A232A912A2322512B87
:1079C0002320612B930B050013840500232C011049
:1079D000232E0110232031132326F1282324D10044
:1079E00017390000130919B7130A5002034B060098
:1079F00063080B3EB3072B0183C7070093041600EF
:107A000093F7870063840706832744006354F004D8
:107A10008327040003C707003307E9000347070073
:107A20001377870063160700138604006FF01FFCAE
:107A30000327C111938717002320F40013071700B1
:107A4000232EE110032744001307F7FF2322E4004D
:107A50006FF09FFB8327C1289305040013850B005B
:107A6000E7800700E30605FA6FF01FFC631A4B116D
:107A7000232A011023260110034716009307A002B2
:107A80006318F700930700012326F11093042600E2
:107A9000938A0400130790009306A00083C50A0090
:107AA00093841A00938705FD637CF7061306300064
:107AB000172500001305C5E7EF00107063040502E9
:107AC000972700009387C7E63305F5408327C11049
:107AD000130710003317A700B3E7E7002326F110C0
:107AE000938A040083C70A001307800793841A004F
:107AF000636EF700130770056362F7041307500203
:107B00006380E7086362F7066386070C930730001B
:107B10002322F1129307A0002328F1106F00801494
:107B200083274111938A0400B387D702938707FD07
:107B3000B387B700232AF1106FF05FF6138787FA37
:107B40001377F70F93060002E3E2E6FC9736000096
:107B500093868692131727003307D7000327070061
:107B60003307D700670007009387B7FB93F7F70F3A
:107B700013072000E36CF7F8930750006F00400AEA
:107B800083274400635AF0028327040003C70700D9
:107B90006318672593871700032744002320F40008
:107BA0008327C1111307F7FF2322E40093871700EF
:107BB000232EF1106FF05FE78327C128930504009F
:107BC00013850B00E7800700E30005FC0325811106
:107BD000631C051C1305F0FF6F00C01D0327C110B7
:107BE000136707022326E1100327C110136707203C
:107BF0002326E110130700012328E1101307E006F4
:107C0000636EF7006F008000232801109307300097
:107C10006F000001930780002328F11093074000B4
:107C20002322F1126F0000041307A0006FF0DFFCA5
:107C30009385040013850900EF00503E8327C1108F
:107C40009304050093E707042326F110930710001F
:107C50006FF01FFD8327C1102322011293E7070451
:107C60002326F110832744006352F00A8327C110B2
:107C700093F70704639E07008327040003C70700E8
:107C80003307E9000347070013778700631C0708E1
:107C900083274112130720006346F70C93068100E7
:107CA000130604009305C11013850B00EF00406814
:107CB000930710006306F51293072000E316F5D62C
:107CC0006FF0DFF0930720006FF09FF58327C1105E
:107CD00013F70701E31A07D40327810093F5170070
:107CE0008326C11113064700638A05002324C100BF
:107CF000832707002390D7006FF01FD32324C100F0
:107D00008327070023A0D7006FF01FD28327C12845
:107D10009305040013850B00E7800700E30805F4D2
:107D20006FF0DFEA0327C11113071700232EE110BC
:107D3000032744001307F7FF2322E4006358E00001
:107D4000938717002320F4006FF01FF38327C128C7
:107D50009305040013850B00E7800700E30E05F090
:107D60006FF0DFE613074000634EF70093068100D3
:107D7000130604009305C11013850B00EF00C073B8
:107D80006FF01FF393070000E38007CA930681009A
:107D9000130604009305C11013850B009700000023
:107DA000E70000006FF0DFF08357C40093F707048B
:107DB000E39207E28320C12B0324812B8324412BF0
:107DC0000329012B8329C12A032A812A832A412AD4
:107DD000032B012A832BC1291301012C678000008A
:107DE000032581116FF01FFD130101FD232E3101C9
:107DF00083A705019309070003A7850023248102B7
:107E00002320210323286101232671012326110247
:107E100023229102232C4101232A5101130B050037
:107E20001384050013090600938B060063D4E70052
:107E3000930707002320F900034734046306070073
:107E4000938717002320F9008327040093F7070284
:107E50006388070083270900938727002320F90000
:107E60008324040093F46400639E0400130A9401C5
:107E7000930AF0FF8327C40003270900B387E74074
:107E800063C4F408832704008346340493F707028D
:107E9000B336D0006392070C1306340493850B00AD
:107EA00013050B00E78009009307F0FF630AF5064E
:107EB00083270400130740009304000093F7670032
:107EC000639EE700832709008324C400B384F44041
:107ED00093C7F4FF93D7F741B3F4F40083278400EA
:107EE000032704016356F700B387E740B384F40027
:107EF000130900001304A401130AF0FF639024097E
:107F0000130500006F0000029306100013060A001C
:107F100093850B0013050B00E7800900631A5503D6
:107F20001305F0FF8320C102032481028324410250
:107F3000032901028329C101032A8101832A410106
:107F4000032B0101832BC100130101036780000093
:107F5000938414006FF01FF23307D400130600035C
:107F6000A301C7040347540493871600B307F40022
:107F700093862600A381E7046FF01FF2930610009A
:107F80001306040093850B0013050B00E78009001E
:107F9000E30845F9130919006FF05FF6130101FCBE
:107FA000232C8102232A91022324410323225103FB
:107FB000232E1102232821032326310383C78501A1
:107FC0009384060093068007130A050013840500B6
:107FD000930A060063E2F602930620061386350430
:107FE00063E0F60263860728930580059726000064
:107FF0009386C694638AB71C130924046F00400457
:108000009386D7F993F6F60F93055001E3E6D5FE74
:10801000972500009385854E93962600B386B6007B
:1080200083A60600B386B600678006008327070094
:10803000130924049386470083A707002320D70051
:108040002301F404930710006F00402683270400E7
:108050000325070093F6070893054500638606028B
:10806000832705002320B70063D807001307D00239
:10807000B307F040A301E404972600009386068C22
:108080001307A0006F00800693F6070483270500FE
:108090002320B700E38A06FC9397070193D7074193
:1080A0006FF09FFC832504008326070013F5050865
:1080B00083A7060093864600631A050093F505041E
:1080C000638605009397070193D707012320D70004
:1080D000834684011307F0066396E6149726000092
:1080E0009386C68513078000A301040483254400FA
:1080F0002324B40063CE050003250400B3E5B700D4
:10810000130906001375B5FF2320A400638405023C
:1081100013090600B3F5E7021309F9FFB385B600AA
:1081200083C505002300B90093850700B3D7E70294
:10813000E3F2E5FE930780006314F702832704004F
:1081400093F71700638E0700032744008327040179
:1081500063C8E70093070003A30FF9FE1309F9FFB3
:10816000330626412328C4001387040093860A009F
:108170001306C1019305040013050A00EFF0DFC6E2
:108180009309F0FF631A35131305F0FF8320C10331
:108190000324810383244103032901038329C102AA
:1081A000032A8102832A410213010104678000002F
:1081B0008327040093E707022320F4009307800736
:1081C000971600009386C678A302F4048325040062
:1081D0000325070013F8050883270500130545004C
:1081E000631A080013F80504630608009397070153
:1081F00093D707012320A70013F715006306070094
:1082000093E505022320B4006386070013070001ED
:108210006FF09FED032704001377F7FD2320E400A0
:108220006FF0DFFE97160000938646711307A000DB
:108230006FF09FEB8326040083270700832544010A
:1082400013F8060813854700630A08002320A700D7
:1082500083A7070023A0B7006F0080012320A70099
:1082600093F6060483A70700E38606FE2390B70073
:1082700023280400130906006FF01FEF832707006F
:108280000326440093050000938647002320D7006F
:1082900003A9070013050900EF000072630605003B
:1082A000330525412322A400832744002328F4001A
:1082B000A30104046FF05FEB832604011306090099
:1082C00093850A0013050A00E7800400E30E35EBEE
:1082D0008327040093F72700639607048327C101CF
:1082E0000325C400E354F5EA138507006FF01FEA85
:1082F0009306100093850A0013050A002326C10087
:10830000E7800400E30235E90326C10013091900E0
:108310008327C4000327C101B387E740E34AF9FC80
:108320006FF0DFFB13090000130694016FF05FFE8E
:1083300083A78500130101FD232481022328610105
:10834000232611022322910223202103232E31010F
:10835000232C4101232A5101130B0500138405002E
:10836000639C070083A78501B337F000B307F04093
:1083700093E7170023A4F5008327040093F7070170
:10838000639A070083A706001387470023A0E6002F
:1083900003A9070093040000130A1000930A2000A9
:1083A000972900009389191B0325840163020504A2
:1083B000631245038327060003C707008327440190
:1083C000B387E70083C70700639407026382040C46
:1083D0006F00C008631455098327060083C7070090
:1083E000B387370183C7070093F7870063980706B1
:1083F000832704009384140093F70701639A07000E
:10840000832706001309190083C70700A30FF9FE8D
:10841000832746009387F7FF2322F6008327060071
:10842000938717002320F600832784009387F7FFA4
:108430002324F4006384070283274600E346F0F612
:10844000832704189305060013050B002326C1009B
:10845000E78007000326C100E30805F48327040032
:1084600093F70701639E07008327C40093871700D3
:108470002326F40083278401638407002300090076
:108480008327040113050000B38797002328F40015
:108490008320C102032481028324410203290102B3
:1084A0008329C101032A8101832A4101032B010190
:1084B0001301010367800000130101FA9717000000
:1084C0009387474A232AF10003A7850197170000E5
:1084D00093878749232CF10097170000938707495A
:1084E000232C81042328210523244105232E7103F5
:1084F000232EF100232E1104232A91042326310573
:108500002322510523206105232C8103232A910373
:108510002328A1032326B1032326A10093073000BB
:108520001384050013090600138A0600970B000048
:10853000938BCB736306F700971B0000938B4B88DC
:10854000832784001307C015130B00009386F7FFE1
:108550006378D700138B37EA9307D0152324F400F0
:108560008327040037170000130707D09309C401BD
:10857000B3E7E7002320F400130C4101938D0900B9
:10858000930A0000930C2000130D100083270900AC
:1085900003250C001306200083C50700EF00C0412F
:1085A00063000508639AAA1383274400639C0700AD
:1085B00083270400930680002322D40093E707203A
:1085C0002320F4008327040093F7F7AF2320F4005F
:1085D000832784009386F7FF2324D4006382070453
:1085E0008327090093841D00938617002320D90058
:1085F00083C707002380FD00832749009387F7FF87
:108600002322F900634CF000832704180325C100DE
:1086100093050900E780070063140518938D040093
:10862000938A1A0093073000130C4C00E390FAF67B
:1086300083254400639605009305A0002322B4001F
:10864000032544019717000093878733B385B7400C
:1086500037FCFFFFEF00801C93840D00930A00009D
:10866000930C0003130CFC6F83278400638E070AAE
:10867000832609000327440103C606003307C70009
:10868000034707006302070A0327040063189607DD
:108690001316470163540606938A1A0063080B00F9
:1086A00093871700130BFBFF2324F4008327490053
:1086B0009387F7FF2322F900635EF0048327090004
:1086C000938717002320F900832784009387F7FFFF
:1086D0002324F4006FF05FF9E39C9AEF83270400F2
:1086E0009306002013F60760E31CD6F29306000100
:1086F0002322D40093E707106FF05FED33778701F3
:108700002320E40083C7060093841400A38FF4FEA3
:108710006FF0DFF9832704180325C10093050900D2
:10872000E7800700E30205FA8327040093F70710A8
:108730006384070263FE990083C5F4FF8327C4178F
:108740000325C100130609009384F4FFE7800700A6
:1087500013051000638634098327040093F707018B
:108760006394070623800400832644000325C10088
:108770001306000093850900E7800B00032704001F
:1087800083270A001376070293864700630E0600CC
:108790002320DA0083A7070023A0A7006F000002B0
:1087A000930A00006FF05FF813761700E30206FEED
:1087B0002320DA0083A707002390A7008327C400A3
:1087C000938717002326F40083270401B3843441E0
:1087D000B3845401B38797002328F40013050000E5
:1087E0008320C10503248105832441050329010554
:1087F0008329C104032A8104832A4104032B010431
:10880000832BC103032C8103832C4103032D01031C
:10881000832DC102130101066780000083C7050094
:108820001307E005638EE7041388150013070000A3
:108830009306000013060010B305D5002380E50061
:1088400093861600E39AC6FE638407041346170056
:108850009308D0021303D0053307F5002300C700A7
:10886000130708008346070013081700638C1603DC
:10887000638C660663800602938706006FF0DFFD57
:1088800083C7150013882500130710006FF05FFAE7
:108890001307F8FF13050700678000009307D00255
:1088A0006FF09FFB83461700938536FAE38805FE39
:1088B000E3C6F6FE1307270093850700938515008E
:1088C0003308B5002300C800E3CAD5FE93050000B5
:1088D00063D6D700B386F6409385F6FF93871700DB
:1088E000B387F5006FF01FF8130708006FF09FFAC9
:1088F000130101FD232481021384050083A5450390
:10890000232611022322910223202103232E310149
:10891000930744046392F50693050040EFE04FBED1
:10892000631205021305F0FF8320C10203248102B4
:1089300083244102032901028329C1011301010398
:108940006780000093070040232CF40283476404EF
:10895000232AA4021305D53F2301F50083475404BD
:10896000A300F500834744042300F5002320A4005E
:10897000130500006FF05FFB832484031399140038
:1089800013060900EF00400993050500E30C05F804
:10899000B30995002326A10013860400138509005E
:1089A000EFE0DF838325C10023203401232C24033F
:1089B000232AB4026FF0DFFB93F5F50F3306C500F1
:1089C0006316C5001305000067800000834705009B
:1089D000E38CB7FE130515006FF09FFE630C0602D3
:1089E0001303050093061000636AB5009306F0FFB9
:1089F0001307F6FF3303E300B385E5008383050027
:108A0000230073001306F6FF3303D300B385D500AC
:108A1000E31606FE678000006396050093050600D6
:108A20006FE00FAE130101FE232C810023244101CE
:108A3000232E1100232A910023282101232631010E
:108A400013040600130A050063180602EFE0CFFEC8
:108A5000930400008320C101032481010329010143
:108A60008329C100032A8100138504008324410166
:108A7000130101026780000093840500EF00C034F9
:108A8000130905006366850093571500E3E487FC2E
:108A90009305040013050A00EFE08FA69309050073
:108AA00063160500938409006FF0DFFA13060400D3
:108AB0006374890013060900938504001385090077
:108AC000EFE0CFF19385040013050A00EFE0CFF645
:108AD0006FF05FFD93B75602638C07001387F6FFB4
:108AE00093870500172300001303D3A6631407021E
:108AF000130101FF23261100EF00802C8320C10009
:108B0000930760012320F500130500001301010104
:108B1000678000009388070003C70700938717004A
:108B2000330867000348080013788800E31408FE40
:108B30001308D0026310070503C70700930F100046
:108B40009387280013F8F6FE631C0804130800033B
:108B5000631E070303C80700930880051378F80D08
:108B60006316180303C717009387270093060001B5
:108B70006F0000031308B002930F0000E31407FD19
:108B800003C70700938728006FF0DFFBE39006FE22
:108B9000130800039306A0006314070193068000E6
:108BA000370E0080130EFEFF338ECF01B372DE024C
:108BB000930800001308000093039000130F900126
:108BC000B35EDE02130307FD63EE630213070300C7
:108BD000635ED70463E80E05938818006384080475
:108BE00063D6E2009308F0FF63880E01930810003B
:108BF00033880603330807019387170003C7F7FF7D
:108C00006FF05FFC1303F7FB63666F00130797FCBD
:108C10006FF01FFC1303F7F9636A6F00130797FAED
:108C20006FF01FFB9308F0FF6FF01FFD1307F0FFBD
:108C3000639EE800130720022320E50013080E00BE
:108C4000631E0600130508006780000063840F00A0
:108C500033080041E30806FE638408009385F7FFAC
:108C60002320B6006FF01FFE6FF0DFE6930F0500C4
:108C700093870500172300001303D38D9388070003
:108C800003C70700938717003305670003480500F3
:108C900013788800E31408FE1305D0026310A704BC
:108CA00003C70700130E10009387280013F5F6FE84
:108CB000631C050413050003631EA70203C8070015
:108CC000130580051378F80D6316A80203C7170073
:108CD00093872700930600016F0000031305B0027D
:108CE000130E0000E314A7FC03C7070093872800B6
:108CF0006FF0DFFBE39006FE130500039306A00070
:108D00006314A700930680001308F0FFB35ED80237
:108D10001305000093029000130F90013373D802E3
:108D200013080000930807FD63F812019308F7FB8E
:108D3000636E1F03930897FC63D6D80463E0AE0408
:108D400013081800630C0802635613011308F0FFA0
:108D50006388AE00130810003387A6023385E8004D
:108D60009387170003C7F7FF6FF0DFFB9308F7F94E
:108D7000636A1F01930897FA6FF01FFC1308F0FF56
:108D80006FF01FFE1307F0FF631CE80013072002BB
:108D900023A0EF0013050800631C06006780000095
:108DA00063040E003305A040630806006304080056
:108DB0009385F7FF2320B600678000006FF01FEB5C
:108DC00003A541926780000083A7C5FF1385C7FFF5
:108DD00063D80700B385A50083A705003305F50018
:048DE00067800000A8
:108DE40049646C65000000000A0D4552524F523A26
:108DF4002076737072696E746628292072657475A2
:108E0400726E206572726F7220636F64653B0A0D27
:108E140000000000D09DD0B5D0B4D0BED181D182A5
:108E2400D0B0D182D0BED187D0BDD18BD0B920D122
:108E340080D0B0D0B7D0BCD0B5D18020D180D0B054
:108E4400D0B1D0BED187D0B5D0B3D0BE20D0B1D1AF
:108E540083D184D0B5D180D0B020D0B4D0BBD18F51
:108E64002076737072696E746628290048454C50E8
:108E7400000000000D2573003F000000D181D0BE2A
:108E8400D185D180D0B0D0BDD0B8D182D18C20D002
:108E9400BDD0B0D181D182D180D0BED0B9D0BAD02A
:108EA400B820D0B220D09FD097D0A30053415645CC
:108EB400434647002025733A2025730A000000002A
:108EC4001B5B303B33316D53746F72652073657473
:108ED40074696E6773202D206661696C6564210A6C
:108EE4004572726F7220636F64653A2025751B5B4F
:108EF400306D0A001B5B303B33326D53746F726507
:108F04002073657474696E6773202D2073756363B1
:108F1400657373211B5B306D0A000000D0B7D0B0BD
:108F2400D0B3D180D183D0B7D0B8D182D18C20D066
:108F3400BDD0B0D181D182D180D0BED0B9D0BAD089
:108F4400B820D0B8D0B720D09FD097D0A3000000CD
:108F54004C4F4144434647001B5B303B33316D4C1F
:108F64006F61642073657474696E6773202D206665
:108F740061696C6564210A4572726F7220636F6463
:108F8400653A2025751B5B306D0A00001B5B303B86
:108F940033326D4C6F61642073657474696E6773EA
:108FA400202D2073756363657373211B5B306D0A19
:108FB40000000000D0B7D0B0D0B3D180D183D0B7F7
:108FC400D0B8D182D18C20D0BDD0B0D181D182D1C2
:108FD40080D0BED0B9D0BAD0B820D0BFD0BE2DD1A9
:108FE40083D0BCD0BED0BBD187D0B0D0BDD0B8D197
:108FF4008E000000444546434647000044656661D0
:10900400756C742073657474696E6773206973205A
:109014006C6F61646564210A00000000D0B2D18BDA
:10902400D0B2D0BED0B420D182D0B5D0BAD183D101
:1090340089D0B8D18520D0BDD0B0D181D182D180A2
:10904400D0BED0B5D0BA00004745544346470000CF
:10905400D186D0B8D0BAD0BBD0B8D187D0B5D18161
:10906400D0BAD0BED0B520D0B2D18BD0BFD0BED074
:10907400BBD0BDD0B5D0BDD0B8D0B520D0BAD0BE4D
:10908400D0BCD0B0D0BDD0B4D18B2C20D0BFD18037
:10909400D0B8D0BCD0B5D1803A206379636C652058
:1090A40031302035302067657420706172616D3114
:1090B4000A092028D0BFD0BED0B2D182D0BED18080
:1090C400D0B8D182D18C20D0BAD0BED0BCD0B0D050
:1090D400BDD0B4D183202267657420706172616D44
:1090E400312220313020D180D0B0D0B720D181209E
:1090F400D0BFD0B0D183D0B7D0BED0B920353020C6
:10910400D0BCD181290000004359434C45000000E4
:1091140025750000D0A16F6D6D616E6420222573EA
:1091240022207265706561742025752074696D65EF
:1091340073207769746820706175736520257520C4
:109144006D73202E2E2E0A00D0BDD0B0D0B7D0BD66
:10915400D0B0D187D0B8D182D18C20D0B3D0BED1F9
:1091640080D18FD187D183D18E20D0BAD0BBD0B05B
:10917400D0B2D0B8D188D183202846312E2E2E46A5
:109184003132292C20D0BFD180D0B8D0BCD0B5D1B9
:10919400803A2062696E64206631207365742070A1
:1091A4006172616D312031323300000042494E4416
:1091B400000000004F6E206B6579202573206269E2
:1091C4006E64656420636F6D6D616E643A2025730F
:1091D4000A000000D0BED182D0BCD0B5D0BDD0B87A
:1091E400D182D18C20D0B3D0BED180D18FD187D1C0
:1091F40083D18E20D0BAD0BBD0B0D0B2D0B8D18871
:10920400D183202846312E2E2E4631322C20616CFB
:109214006C202D20D0B2D181D0B520D181D180D085
:10922400B0D0B7D183292C20D0BFD180D0B8D0BC46
:10923400D0B5D1803A20756E62696E6420663100C3
:10924400554E42494E440000414C4C004B65792038
:109254002573202D20756E62696E646564210A0091
:10926400416C6C206B65797320756E62696E646500
:1092740064210A001B5B324B0D0000000D25732591
:10928400730000001B5B43001B5B44001B5B2575E4
:10929400440000000D257325730A00001B5B25752F
:1092A4004300000025732008000000000820080087
:1092B40008257320080000002573000046310000D3
:1092C40046320000463300004634000046350000B4
:1092D4004636000046370000463800004639000094
:1092E4004631300046313100463132001B5B303BA1
:1092F40033356D43534B593E1B5B306D000000000A
:10930400747374313A20202575202D2025730A00AA
:10931400747374323A20202575202D2025730A0099
:10932400747374333A20202575202D2025730A0088
:109334003E3E202025730A00203C3C2025730A0071
:109344004F4B0000494D45493A2025730A0000005F
:109354001B5B303B33316D4368616E67652062612E
:10936400756472617465206F6E202575211B5B30F6
:109374006D0A00004552524F523A2066775F6C6581
:109384006E203D2025750A0041540D001B5B303BC7
:1093940033326D4154202D204F4B1B5B306D0A003E
:1093A40041542B4347534E0D000000001B5B303BE0
:1093B40033316D4552524F523A20696D65692063CD
:1093C4006865636B206469676974206572726F7283
:1093D400211B5B306D0A00001B5B303B33326D494F
:1093E4004D454920636865636B202D204F4B1B5B03
:1093F400306D0A002B43455245473A20302C31004A
:109404002B43455245473A20302C350041542B43D9
:10941400455245473F0D00001B5B303B33326D4CDA
:109424005445202D20636F6E6E6563746564211B43
:109434005B306D0A000000001B5B303B33326D4C27
:109444005445202D20636F6E6E65637465642069D6
:109454006E20726F616D696E67211B5B306D0A004F
:109464002B43475245473A20302C31002B43475277
:1094740045473A20302C350041542B434752454749
:109484003F0D00001B5B303B33326D47505253207D
:109494002D20636F6E6E6563746564211B5B306D94
:1094A4000A0000001B5B303B33326D47505253209F
:1094B4002D20636F6E6E656374656420696E20721F
:1094C4006F616D696E67211B5B306D0A00000000DF
:1094D40041542B5A495043414C4C3D310D0000003E
:1094E40041542B434744434F4E543D312C22495061
:1094F400222C22434D4E4554220D000041542B5A38
:1095040049504F50454E3D312C312C2273746167C4
:10951400652E6169722D6C696E6B2E737061636563
:10952400222C31303030302C353030300D000000FA
:109534002B5A4950535441543A312C310000000005
:109544001B5B303B33326D536572766572202D2080
:10955400636F6E6E6563746564211B5B306D0A0016
:10956400434F4E4E4543540041542B5A49504352A5
:10957400454154453D310D001B5B303B33326D5248
:109584006177206D6F6465202D2061637469766155
:10959400746564211B5B306D0A00000041542B5A32
:1095A4004950434C4F53453D310D000041542B5A13
:1095B400495043414C4C3D300D00000041757468E6
:1095C400656E74696669636174696F6E2E2E2E0A06
:1095D400000000001B5B303B33326D5452414E534C
:1095E400504152454E54211B5B306D0A000000006F
:1095F4004669726D7761726520646F776E6C6F6116
:10960400642E2E2E0A000000656E640A000000001D
:109614001B5B303B33316D48656172744265617424
:109624002074696D656F757421206474696D65209B
:109634003D2025751B5B306D0A00000061745F746A
:10964400785F6275663A2025750A000061745F725E
:10965400785F6275663A2025750A000041545F728E
:109664006573706F6E73655F636865636B28293A11
:1096740020696E76616C6964207265737020666F10
:10968400726D6174210000006578745F74785F62A4
:1096940075663A2025750A006578745F72785F6292
:1096A40075663A2025750A006E6F742070757368AC
:1096B400656400002073657420706172616D657467
:1096C40065720000534554005453543100000000A7
:1096D400747374313A20000020656E746572656499
:1096E4003A2025750A0000002067657420706172B5
:1096F400616D65746572000047455400207072699D
:109704006E7420696E666F206F6620646576697377
:10971400652073746174650053544154450000001E
:1097240073746174653A2025750A000042494E44F9
:109734003A2025730A000000737461745F61745FDA
:1097440074785F636E743A2025750A0073746174CB
:109754005F61745F72785F636E743A2025750A00E6
:10976400737461745F6578745F74785F636E743A60
:109774002025750A00000000737461745F657874B5
:109784005F72785F636E743A2025750A00000000EA
:10979400737461745F6D61766C696E6B5F66726120
:1097A4006D655F6572725F636E743A2025750A0099
:1097B400207072696E7420736F66742064617465BE
:1097C40000000000534F4654000000004D61792012
:1097D4002036203230323600536F66742064617450
:1097E400653A2025730A0000535441434B0000009E
:1097F4000A1B5B303B33316DD09ED0A8D098D091FA
:10980400D09AD0903A2025731B5B306D0A0000007B
:109814000A4D432069732073746172746564206F08
:109824006E2025752C25303375204D487A210A0089
:10983400D097D0B0D0B3D180D183D0B6D0B5D0BD7D
:10984400D18B20D0BDD0B0D181D182D180D0BED037
:10985400B9D0BAD0B820D0BFD0BE20D183D0BCD02C
:10986400BED0BBD187D0B0D0BDD0B8D18E210A0034
:10987400D0A0D0B0D0B7D0BCD0B5D18020D181D0C9
:10988400B2D0BED0B1D0BED0B4D0BDD0BED0B3D093
:10989400BE20D0BFD180D0BED181D182D180D0B002
:1098A400D0BDD181D182D0B2D0B020D181D182D0EB
:1098B400B5D0BAD0BED0B220D0BFD180D0BED18670
:1098C400D0B5D181D181D0BED0B22028D0B1D0B012
:1098D400D0B9D182293A0A0050726F635F4D616931
:1098E4006E3A2025750A000050726F635F434C493D
:1098F4003A2025750A0000000A1B5B313B33316DA9
:109904004865617020616E6420737461636B2063C9
:109914006F6C6C6973696F6E211B5B306D0A00009C
:10992400232D302B20000000686C4C0065666745D1
:109934004647000030313233343536373839414206
:109944004344454600000000303132333435363765
:109954003839616263646566000000002B2D0000E5
:109964003030000078580000412D46612D663839AA
:1099740030313233343536375D0000000000891150
:1099840012239B322446AD573665BF74488CC19D63
:109994005AAFD3BE6CCAE5DB7EE9F7F88110080143
:1099A40093331A22A5562C47B7753E64C99C408D43
:1099B400DBBF52AEEDDA64CBFFF976E802218B30DF
:1099C400100299132667AF763444BD554AADC3BC23
:1099D400588ED19F6EEBE7FA7CC8F5D983310A2003
:1099E40091121803A7772E66B5543C45CBBD42AC03
:1099F400D99E508FEFFB66EAFDD874C904428D539B
:109A040016619F702004A9153227BB364CCEC5DFE2
:109A14005EEDD7FC6888E1997AABF3BA85520C43C2
:109A240097711E60A1142805B3373A26CDDE44CFC2
:109A3400DFFD56ECE9986089FBBB72AA06638F725E
:109A440014409D512225AB343006B9174EEFC7FEA2
:109A54005CCCD5DD6AA9E3B8788AF19B87730E6282
:109A640095501C41A3352A24B1163807CFFF46EE82
:109A7400DDDC54CDEBB962A8F99A708B088481952A
:109A84001AA793B62CC2A5D33EE1B7F04008C91972
:109A9400522BDB3A644EED5F766DFF7C8994008532
:109AA4009BB712A6ADD224C3BFF136E0C118480952
:109AB400D33B5A2AE55E6C4FF77D7E6C0AA583B4CE
:109AC400188691972EE3A7F23CC0B5D14229CB3832
:109AD400500AD91B666FEF7E744CFD5D8BB502A4F2
:109AE40099961087AFF326E2BDD034C1C3394A2812
:109AF400D11A580BE77F6E6EF55C7C4D0CC685D78A
:109B04001EE597F42880A1913AA3B3B2444ACD5BF1
:109B14005669DF78600CE91D722FFB3E8DD604C7B1
:109B24009FF516E4A9902081BBB332A2C55A4C4BD1
:109B3400D7795E68E11C680DF33F7A2E0EE787F64D
:109B44001CC495D52AA1A3B03882B193466BCF7AB1
:109B54005448DD59622DEB3C700EF91F8FF706E671
:109B64009DD414C5ABB122A0B9923083C77B4E6A91
:109B7400D5585C49E33D6A2CF11E780F1C27008000
:109B8400DC2700807C280080442800808025008019
:109B9400802500808025008080250080802500802D
:109BA400802500808025008080250080802500801D
:109BB400802500808025008080250080F425008099
:109BC40078260080B8260080DA2600808025008070
:109BD400622800808025008002270080D42700802E
:109BE400D0270080CC270080C8270080C4270080AD
:109BF40080250080C0270080D82700807C27008033
:109C04000D1B5B303B33316D496E76616C696420AA
:109C14006B6579776F7264211B5B306D0A000000FD
:109C24000AD0A1D09FD0A0D090D092D09AD0900A40
:109C34000AD09FD0A0D090D092D098D09BD0902022
:109C4400D097D090D09FD098D0A1D09820D09AD03F
:109C54009ED09CD090D09DD0943A0A202E2E2E20B7
:109C64002D20D0BDD0B020D0BCD0B5D181D182D0F0
:109C7400B520D0BCD0BDD0BED0B3D0BED182D0BE72
:109C8400D187D18CD18F20D0B4D0BED0BBD0B6D0A8
:109C9400BDD0B020D0B1D18BD182D18C20D0BED058
:109CA400B4D0BDD0B020D0B8D0B720D0BFD0B5D1BB
:109CB40080D0B5D187D0B8D181D0BBD0B5D0BDD0FC
:109CC400BDD18BD18520D0BDD0B8D0B6D0B520D0F1
:109CD400BAD0BED0BCD0B0D0BDD0B42E0A20287724
:109CE4002C20752C20782C20792C20752C207A2976
:109CF400202D20D0BCD0BED0B6D0B5D18220D0B1DA
:109D0400D18BD182D18C20D182D0BED0BBD18CD08A
:109D1400BAD0BE20D0BED0B4D0B8D0BD20D0B8D038
:109D2400B720D0BFD0B5D180D0B5D187D0B8D1813C
:109D3400D0BBD0B5D0BDD0BDD18BD18520D0B20A97
:109D44000920D0BAD180D183D0B3D0BBD18BD185F7
:109D540020D181D0BAD0BED0B1D0BAD0B0D1852074
:109D6400D187D0B5D180D0B5D0B720D0B7D0B0D0BE
:109D7400BFD18FD182D183D18E20D0BFD0B0D1803A
:109D8400D0B0D0BCD0B5D182D180D0BED0B220D09A
:109D9400B8D0BBD0B820D0BAD0BED0BCD0B0D0BD23
:109DA400D0B42E0A207B787D202D20D0B220D184FF
:109DB400D0B8D0B3D183D180D0BDD18BD18520D1BF
:109DC40081D0BAD0BED0B1D0BAD0B0D18520D183A1
:109DD400D0BAD0B0D0B7D18BD0B2D0B0D18ED182DE
:109DE400D181D18F20D0BDD0B5D0BED0B1D18FD04C
:109DF400B7D0B0D182D0B5D0BBD18CD0BDD18BD0AF
:109E0400B520D0BFD0B0D180D0B0D0BCD0B5D18235
:109E1400D180D18B2E0A205B782E2E585D202D20E8
:109E2400D0B220D0BFD180D18FD0BCD0BED183D00E
:109E3400B3D0BED0BBD18CD0BDD18BD18520D18144
:109E4400D0BAD0BED0B1D0BAD0B0D18520D183D0D1
:109E5400BAD0B0D0B7D18BD0B2D0B0D0B5D182D136
:109E640081D18F20D0B4D0B8D0B0D0BFD0B0D0B7CB
:109E7400D0BED0BD20D0B4D0BED0BFD183D181D18B
:109E840082D0B8D0BCD18BD18520D0B7D0BDD0B0D2
:109E9400D187D0B5D0BDD0B8D0B920D0B4D0BBD143
:109EA4008F20D187D0B8D181D0BBD0B02C0A092063
:109EB400D0BFD0BED0B4D181D182D0B0D0B2D0BBCB
:109EC400D18FD0B5D0BCD0BED0B3D0BE20D0B220BC
:109ED400D0BAD0BED0BCD0B0D0BDD0B4D18320D005
:109EE400BDD0B020D18DD182D0BED0BC20D0BCD0CA
:109EF400B5D181D182D0B52E0A0AD09AD09ED09CF9
:109F0400D090D09DD094D0AB3A0A0000D182D0B585
:109F1400D181D182D0BED0B2D18BD0B920D0BFD024
:109F2400B0D180D0B0D0BCD0B5D182D180203300A4
:109F3400D182D0B5D181D182D0BED0B2D18BD0B9AB
:109F440020D0BFD0B0D180D0B0D0BCD0B5D182D1D8
:109F540080203200D182D0B5D181D182D0BED0B29E
:109F6400D18BD0B920D0BFD0B0D180D0B0D0BCD0AC
:109F7400B5D182D18020310052096AD53036A53856
:109F8400BF40A39E81F3D7FB7CE339829B2FFF87DD
:109F9400348E4344C4DEE9CB547B9432A6C2233DC1
:109FA400EE4C950B42FAC34E082EA16628D924B272
:109FB400765BA2496D8BD12572F8F6648668981693
:109FC400D4A45CCC5D65B6926C704850FDEDB9DAF2
:109FD4005E154657A78D9D8490D8AB008CBCD30AE0
:109FE400F7E45805B8B34506D02C1E8FCA3F0F02BC
:109FF400C1AFBD0301138A6B3A9111414F67DCEA8B
:10A0040097F2CFCEF0B4E67396AC7422E7AD358503
:10A01400E2F937E81C75DF6E47F11A711D29C5890D
:10A024006FB7620EAA18BE1BFC563E4BC6D27920EF
:10A034009ADBC0FE78CD5AF41FDDA8338807C731F8
:10A04400B11210592780EC5F60517FA919B54A0DF0
:10A054002DE57A9F93C99CEFA0E03B4DAE2AF5B065
:10A06400C8EBBB3C83539961172B047EBA77D62681
:10A07400E169146355210C7D637C777BF26B6FC5BA
:10A084003001672BFED7AB76CA82C97DFA5947F0F7
:10A09400ADD4A2AF9CA472C0B7FD9326363FF7CCD3
:10A0A40034A5E5F171D8311504C723C31896059A70
:10A0B400071280E2EB27B27509832C1A1B6E5AA093
:10A0C400523BD6B329E32F8453D100ED20FCB15B7E
:10A0D4006ACBBE394A4C58CFD0EFAAFB434D3385E7
:10A0E40045F9027F503C9FA851A3408F929D38F5BB
:10A0F400BCB6DA2110FFF3D2CD0C13EC5F974417F2
:10A10400C4A77E3D645D197360814FDC222A908868
:10A1140046EEB814DE5E0BDBE0323A0A4906245CF4
:10A12400C2D3AC629195E479E7C8376D8DD54EA959
:10A134006C56F4EA657AAE08BA78252E1CA6B4C625
:10A14400E8DD741F4BBD8B8A703EB5664803F60E7E
:10A15400613557B986C11D9EE1F8981169D98E946D
:10A164009B1E87E9CE5528DF8CA1890DBFE6426886
:10A1740041992D0FB054BB16DA3A0080DA3A0080C8
:10A18400BA3B0080E23B0080083C0080143C008025
:10A19400223C0080303C00803E3C0080663C0080D5
:10A1A4009C3C0080D03C0080F83C00809E3D0080B8
:10A1B4009E3D00801E3E0080401F00009002020071
:10A1C40000000000411F00004E81810000000000DB
:10A1D400421F0000CA10100000000000431F0000CE
:10A1E4002C01010000000000441F00008809090040
:10A1F40000000000451F00001C08080000000000CB
:10A20400461F00006601010000000000982F8A42EA
:10A2140091443771CFFBC0B5A5DBB5E95BC25639B4
:10A22400F111F159A4823F92D55E1CAB98AA07D8CC
:10A23400015B8312BE853124C37D0C55745DBE72EF
:10A24400FEB1DE80A706DC9B74F19BC1C1699BE46F
:10A254008647BEEFC69DC10FCCA10C246F2CE92DFF
:10A26400AA84744ADCA9B05CDA88F97652513E9823
:10A274006DC631A8C82703B0C77F59BFF30BE0C62A
:10A284004791A7D55163CA0667292914850AB727B8
:10A2940038211B2EFC6D2C4D130D385354730A6555
:10A2A400BB0A6A762EC9C281852C7292A1E8BFA22C
:10A2B4004B661AA8708B4BC2A3516CC719E892D194
:10A2C400240699D685350EF470A06A1016C1A41917
:10A2D400086C371E4C774827B5BCB034B30C1C3916
:10A2E4004AAAD84E4FCA9C5BF36F2E68EE828F74D5
:10A2F4006F63A5781478C8840802C78CFAFFBE90EF
:10A30400EB6C50A4F7A3F9BEF27871C6D182D0B534
:10A31400D181D182D0BED0B2D18BD0B920D0BFD020
:10A32400B0D180D0B0D0BCD0B5D182D180203100A2
:10A334000D1B5B303B33316D496E76616C69642073
:10A344006B6579776F7264211B5B306D0A000000C6
:10A354000D1B5B303B33316D556E6B6E6F776E202A
:10A36400636F6D6D616E64211B5B306D0A000000CC
:10A3740000010202030303030404040404040404A8
:10A384000505050505050505050505050505050579
:10A394000606060606060606060606060606060659
:10A3A4000606060606060606060606060606060649
:10A3B4000707070707070707070707070707070729
:10A3C4000707070707070707070707070707070719
:10A3D4000707070707070707070707070707070709
:10A3E40007070707070707070707070707070707F9
:10A3F40008080808080808080808080808080808D9
:10A4040008080808080808080808080808080808C8
:10A4140008080808080808080808080808080808B8
:10A4240008080808080808080808080808080808A8
:10A434000808080808080808080808080808080898
:10A444000808080808080808080808080808080888
:10A454000808080808080808080808080808080878
:10A464000808080808080808080808080808080868
:10A4740074D7FFFF98D6FFFF98D6FFFFBCD7FFFF26
:10A4840098D6FFFF98D6FFFF98D6FFFF98D6FFFF18
:10A4940098D6FFFF98D6FFFF98D6FFFFE0D7FFFFBF
:10A4A400B4D7FFFF04D7FFFF04D7FFFF04D7FFFF94
:10A4B40098D6FFFF94D7FFFF98D6FFFF98D6FFFFEB
:10A4C40098D6FFFF98D6FFFF58D8FFFFA0D7FFFF0D
:10A4D40068D7FFFF98D6FFFF98D6FFFF50D8FFFF3D
:10A4E40098D6FFFFB4D7FFFF98D6FFFF98D6FFFF9B
:10A4F40074D7FFFF34DBFFFF54DBFFFF00DBFFFFFC
:10A5040000DBFFFF00DBFFFF00DBFFFF54DBFFFF8F
:10A5140000DBFFFF00DBFFFF00DBFFFF00DBFFFFD3
:10A524003CDDFFFFACDBFFFFB8DCFFFF00DBFFFF20
:10A5340000DBFFFF84DDFFFF00DBFFFFACDBFFFF81
:10A5440000DBFFFF00DBFFFFC4DCFFFF0020202057
:10A5540020202020202028282828282020202020CF
:10A56400202020202020202020202020208810109F
:10A5740010101010101010101010101010040404FB
:10A5840004040404040404101010101010104141B9
:10A5940041414141010101010101010101010101A7
:10A5A40001010101010101011010101010104242BB
:10A5B4004242424202020202020202020202020277
:10A5C4000202020202020202101010102000000017
:10A5D4000000000000000000000000000000000077
:10A5E4000000000000000000000000000000000067
:10A5F4000000000000000000000000000000000057
:10A604000000000000000000000000000000000046
:10A614000000000000000000000000000000000036
:10A624000000000000000000000000000000000026
:10A634000000000000000000000000000000000016
:0DA644000000000000000000000000000009
:10A6540003041800401D00801C1A0080482000805C
:10A664000E1E00808D01020408102040801B36005D
:10A6740041542B5A5253540D000000002A7E2516D3
:0CA6840038AED2A67BF7558809CF5F3CAA
:10A6900000000000562F00805C2F0080682F008093
:10A6A000C00F0080060000000101000000C2010090
:10A6B00000C20100000000000000000000000000D7
:10A6C00002000000000000008C11C16F421703005F
:10A6D0000000010000000000184700402802004070
:10A6E000000000000000000000000000000000006A
:10A6F000000000000000000000000000000000005A
:10A700000000000000000000000000000000000049
:10A710000000000000000000000000000000000039
:10A720000000000000000000000000000000000029
:10A730000000000000000000000000000000000019
:10A740000000000000000000000000000000000009
:10A7500000000000000000000000000000000000F9
:10A7600000000000000000000000000000000000E9
:10A7700000000000000000000000000000000000D9
:10A7800000000000000000000000000000000000C9
:10A7900000000000000000000000000000000000B9
:10A7A00000000000000000000000000000000000A9
:10A7B0000000000000000000000000000000000099
:10A7C0000000000000000000000000000000000089
:10A7D0000000000000000000000000000000000079
:10A7E00000000000A04100400842004070420040CC
:10A7F0000000000000000000000000000000000059
:10A800000000000000000000000000000000000048
:10A810000000000000000000000000000000000038
:0CA820000000000000000000000000002C
:040000058000000077
:00000001FF
